 RT2870

 Timestamp is 4b18d4d5 (Fri Dec 04 17:22:29 2009)

 Preferred load address is 10000000

 Start         Length     Name                   Class
 0001:00000000 00009681H .rdata                  CODE
 0001:00009684 00000023H .rdata$debug            CODE
 0001:000096a8 0008bc60H .text                   CODE
 0001:00095308 0000039cH .xdata                  CODE
 0001:000956a4 0000003cH .idata$2                CODE
 0001:000956e0 00000014H .idata$3                CODE
 0001:000956f4 00000148H .idata$4                CODE
 0001:0009583c 000004c4H .idata$6                CODE
 0001:00095d00 0000009bH .edata                  CODE
 0002:00000000 00000148H .idata$5                DATA
 0002:00000148 0000a39cH .data                   DATA
 0002:0000a500 00003ee0H .bss                    DATA
 0003:00000000 00001b80H .pdata                  DATA

  Address         Publics by Value              Rva+Base       Lib:Object

 0000:00000000       ___safe_se_handler_table   00000000     <absolute>
 0000:00000000       ___safe_se_handler_count   00000000     <absolute>
 0001:00000620       ??_C@_0CM@OBCIMEMP@has?5disassociated?5with?5invalid?5P@ 10001620     ap.obj
 0001:0000064c       ??_C@_0BH@IGJNPKB@active?5countermeasures?$AA@ 1000164c     ap.obj
 0001:00000664       ??_C@_0CE@JFLNOENI@has?5been?5aged?9out?5and?5disassocia@ 10001664     ap.obj
 0001:00000688       ??_C@_0BC@HLHDIMIG@has?5disassociated?$AA@ 10001688     ap.obj
 0001:0000069c       ??_C@_0BI@ICOOKKNB@successfully?5associated?$AA@ 1000169c     ap.obj
 0001:000006b4       ??_C@_0BF@ILIMBFOC@restart?5access?5point?$AA@ 100016b4     ap.obj
 0001:000008d0       ??_C@_05GCOINAMN@My?5AP?$AA@ 100018d0     ap.obj
 0001:00001cd8       ISbox                      10002cd8     Ap_wapi.obj
 0001:00001dd8       ??_C@_0FD@HHMGDLDH@multicast?5or?5station?5key?5expansi@ 10002dd8     Ap_wapi.obj
 0001:00001e2c       ??_C@_0DP@OEHPIDIO@preshared?5key?5expansion?5for?5auth@ 10002e2c     Ap_wapi.obj
 0001:00001e70       ??_C@_0EB@FIKGLGCJ@pairwise?5key?5expansion?5for?5unica@ 10002e70     Ap_wapi.obj
 0001:00001eb4       ??_C@_0L@PNLLBLCL@1234567890?$AA@ 10002eb4     Ap_wapi.obj
 0001:00002ac0       ??_C@_0CB@BBPBGEJA@IEEE802?411?5WIRELESS?5ACCESS?5POINT@ 10003ac0     dls.obj
 0001:00003208       ??_C@_0N@BOOJCAPA@HW?5Diversity?$AA@ 10004208     mlme.obj
 0001:00003218       ??_C@_05LKLMIBEG@Ant?9B?$AA@ 10004218     mlme.obj
 0001:00003220       ??_C@_05JBJBNCIF@Ant?9A?$AA@ 10004220     mlme.obj
 0001:00003228       ??_C@_0N@ENCHDJIJ@SW?5Diversity?$AA@ 10004228     mlme.obj
 0001:00003238       ??_C@_0DC@DNIOBKKO@4?9way?5handshake?5IE?5diff?5among?5As@ 10004238     mlme.obj
 0001:0000326c       ??_C@_0CE@ODBDOOLB@2?9way?5?$CIgroup?5key?$CJ?5handshake?5time@ 1000426c     mlme.obj
 0001:00003290       ??_C@_0BI@IFDLABDB@4?9way?5handshake?5timeout?$AA@ 10004290     mlme.obj
 0001:000032a8       ??_C@_09CJDAIAGP@MIC?5error?$AA@ 100042a8     mlme.obj
 0001:000032b4       ??_C@_0L@LCBPMDKI@invalid?5IE?$AA@ 100042b4     mlme.obj
 0001:000032c0       ??_C@_0CD@EMJAOFKL@require?5auth?5before?5assoc?1re?9ass@ 100042c0     mlme.obj
 0001:000032e4       ??_C@_0O@IBGJFIPI@class?53?5error?$AA@ 100042e4     mlme.obj
 0001:000032f4       ??_C@_0O@ENMDFIGG@class?52?5error?$AA@ 100042f4     mlme.obj
 0001:00003304       ??_C@_0CE@IOCPNGNK@AP?5unable?5to?5hanle?5all?5associati@ 10004304     mlme.obj
 0001:00003328       ??_C@_0BM@OBHJDPBG@DIS?9ASSOC?5due?5to?5inactivity?$AA@ 10004328     mlme.obj
 0001:00003344       ??_C@_0BK@BAGFOGKD@STA?5is?5leaving?5?1?5has?5left?$AA@ 10004344     mlme.obj
 0001:00003360       ??_C@_0BO@PEBKGJDA@Previous?5Auth?5no?5longer?5valid?$AA@ 10004360     mlme.obj
 0001:00003380       ??_C@_0BD@PBGFPAEA@Unspecified?5Reason?$AA@ 10004380     mlme.obj
 0001:00003394       ??_C@_08NKCLJDKG@Reserved?$AA@ 10004394     mlme.obj
 0001:000035a0       ??_C@_00CNPNBAHC@?$AA@     100045a0     mlme.obj
 0001:00003bc4       ??_C@_1BE@GIGCBHND@?$AAC?$AAh?$AA1?$AA4?$AAB?$AAO?$AAn?$AAl?$AAy?$AA?$AA@ 10004bc4     rtmp_init.obj
 0001:00003bd8       ??_C@_1CA@MPGMFPNC@?$AAB?$AAT?$AAC?$AAo?$AAn?$AAf?$AAi?$AAg?$AAu?$AAr?$AAa?$AAt?$AAi?$AAo?$AAn?$AA?$AA@ 10004bd8     rtmp_init.obj
 0001:00003bf8       ??_C@_1BK@CJJNEDPG@?$AAB?$AAT?$AAS?$AAo?$AAf?$AAt?$AAw?$AAa?$AAr?$AAe?$AAO?$AAn?$AA?$AA@ 10004bf8     rtmp_init.obj
 0001:00003c14       ??_C@_1BK@BABIKIEF@?$AAG?$AAa?$AAi?$AAn?$AAP?$AAr?$AAo?$AAS?$AAp?$AAe?$AAe?$AAd?$AA?$AA@ 10004c14     rtmp_init.obj
 0001:00003c30       ??_C@_1CC@GCNEADEG@?$AAB?$AAs?$AAs?$AAi?$AAd?$AAR?$AAe?$AAp?$AAo?$AAs?$AAi?$AAt?$AAT?$AAi?$AAm?$AAe?$AA?$AA@ 10004c30     rtmp_init.obj
 0001:00003c54       ??_C@_1CC@KKEIICNE@?$AAP?$AAr?$AAo?$AAh?$AAi?$AAb?$AAi?$AAt?$AAT?$AAK?$AAI?$AAP?$AAo?$AAn?$AAH?$AAT?$AA?$AA@ 10004c54     rtmp_init.obj
 0001:00003c78       ??_C@_19EIBINHIL@?$AAW?$AAA?$AAP?$AAI?$AA?$AA@ 10004c78     rtmp_init.obj
 0001:00003c84       ??_C@_19DICJPJO@?$AAT?$AAE?$AAS?$AAT?$AA?$AA@ 10004c84     rtmp_init.obj
 0001:00003c90       ??_C@_1BO@LFECHPJM@?$AAC?$AAo?$AAu?$AAn?$AAt?$AAr?$AAy?$AAT?$AAx?$AAP?$AAw?$AAr?$AA5?$AAG?$AA?$AA@ 10004c90     rtmp_init.obj
 0001:00003cb0       ??_C@_1BK@ENDJOIGJ@?$AAC?$AAo?$AAu?$AAn?$AAt?$AAr?$AAy?$AAT?$AAx?$AAP?$AAw?$AAr?$AA?$AA@ 10004cb0     rtmp_init.obj
 0001:00003ccc       ??_C@_1BI@LGPNEEJB@?$AAL?$AAE?$AAD?$AAP?$AAo?$AAl?$AAa?$AAr?$AAi?$AAt?$AAy?$AA?$AA@ 10004ccc     rtmp_init.obj
 0001:00003ce4       ??_C@_1O@PFJDAPJC@?$AAL?$AAE?$AAD?$AAA?$AAc?$AAt?$AA?$AA@ 10004ce4     rtmp_init.obj
 0001:00003cf4       ??_C@_1BE@IFGCHPPB@?$AAL?$AAE?$AAD?$AAC?$AAo?$AAn?$AAf?$AAi?$AAg?$AA?$AA@ 10004cf4     rtmp_init.obj
 0001:00003d08       ??_C@_1BA@JBHFPAPB@?$AAL?$AAE?$AAD?$AAM?$AAo?$AAd?$AAe?$AA?$AA@ 10004d08     rtmp_init.obj
 0001:00003d18       ??_C@_1BG@PLJAEAAM@?$AAL?$AAE?$AAD?$AAC?$AAt?$AAl?$AAB?$AAy?$AAS?$AAW?$AA?$AA@ 10004d18     rtmp_init.obj
 0001:00003d30       ??_C@_1CA@LJPPBOF@?$AAL?$AAi?$AAn?$AAk?$AAS?$AAp?$AAe?$AAe?$AAd?$AAS?$AAt?$AAa?$AAt?$AAu?$AAs?$AA?$AA@ 10004d30     rtmp_init.obj
 0001:00003d50       ??_C@_1DC@LFKLGNPI@?$AAS?$AAo?$AAf?$AAt?$AAA?$AAP?$AAF?$AAo?$AAr?$AAc?$AAe?$AAM?$AAu?$AAl?$AAt?$AAi?$AAc?$AAa?$AAs?$AAt?$AAR?$AAa?$AAt?$AAe?$AA?$AA@ 10004d50     rtmp_init.obj
 0001:00003d84       ??_C@_1BC@OGAKBKDE@?$AAI?$AAd?$AAl?$AAe?$AAT?$AAi?$AAm?$AAe?$AA?$AA@ 10004d84     rtmp_init.obj
 0001:00003d98       ??_C@_1BG@IINBLCLB@?$AAD?$AAt?$AAi?$AAm?$AAP?$AAe?$AAr?$AAi?$AAo?$AAd?$AA?$AA@ 10004d98     rtmp_init.obj
 0001:00003db0       ??_C@_1CE@PCANMBOM@?$AAA?$AAu?$AAt?$AAo?$AAC?$AAh?$AAa?$AAn?$AAn?$AAe?$AAl?$AAS?$AAe?$AAl?$AAe?$AAc?$AAt?$AA?$AA@ 10004db0     rtmp_init.obj
 0001:00003dd4       ??_C@_1BE@NOKFBOKB@?$AAP?$AAS?$AAC?$AAo?$AAn?$AAt?$AAr?$AAo?$AAl?$AA?$AA@ 10004dd4     rtmp_init.obj
 0001:00003de8       ??_C@_1BE@DBKPDCJJ@?$AAS?$AAm?$AAa?$AAr?$AAt?$AAS?$AAc?$AAa?$AAn?$AA?$AA@ 10004de8     rtmp_init.obj
 0001:00003dfc       ??_C@_1BE@IINHAOJL@?$AAR?$AAs?$AAs?$AAi?$AAD?$AAe?$AAl?$AAt?$AAa?$AA?$AA@ 10004dfc     rtmp_init.obj
 0001:00003e10       ??_C@_1CI@CFGDGLJB@?$AAC?$AAC?$AAX?$AAP?$AAk?$AAt?$AAL?$AAo?$AAs?$AAs?$AAL?$AAi?$AAm?$AAi?$AAt?$AAT?$AAi?$AAm?$AAe?$AA?$AA@ 10004e10     rtmp_init.obj
 0001:00003e38       ??_C@_1CA@KIMCJOKE@?$AAC?$AAA?$AAC?$AAD?$AAr?$AAo?$AAp?$AAC?$AAr?$AAi?$AAt?$AAe?$AAr?$AAi?$AAa?$AA?$AA@ 10004e38     rtmp_init.obj
 0001:00003e58       ??_C@_1BM@PHBOPLGB@?$AAC?$AAA?$AAC?$AAD?$AAr?$AAo?$AAp?$AAP?$AAe?$AAr?$AAi?$AAo?$AAd?$AA?$AA@ 10004e58     rtmp_init.obj
 0001:00003e74       ??_C@_1BK@PJKHDBMG@?$AAC?$AAC?$AAX?$AAD?$AAb?$AAm?$AAO?$AAf?$AAf?$AAs?$AAe?$AAt?$AA?$AA@ 10004e74     rtmp_init.obj
 0001:00003e90       ??_C@_1BC@GBGBNBCD@?$AAC?$AAL?$AAF?$AAa?$AAc?$AAt?$AAo?$AAr?$AA?$AA@ 10004e90     rtmp_init.obj
 0001:00003ea4       ??_C@_1BC@EGPLFCEP@?$AAN?$AAH?$AAF?$AAa?$AAc?$AAt?$AAo?$AAr?$AA?$AA@ 10004ea4     rtmp_init.obj
 0001:00003eb8       ??_C@_1BI@GKAHDKBF@?$AAC?$AAC?$AAX?$AA2?$AAC?$AAo?$AAn?$AAt?$AAr?$AAo?$AAl?$AA?$AA@ 10004eb8     rtmp_init.obj
 0001:00003ed0       ??_C@_1O@LPLILBCD@?$AAP?$AAS?$AAM?$AAo?$AAd?$AAe?$AA?$AA@ 10004ed0     rtmp_init.obj
 0001:00003ee0       ??_C@_1CO@GMOLFAC@?$AAA?$AAd?$AAh?$AAo?$AAc?$AAN?$AA1?$AA4?$AAC?$AAh?$AA4?$AA0?$AAM?$AAH?$AAz?$AAA?$AAl?$AAl?$AAo?$AAw?$AAe?$AAd?$AA?$AA@ 10004ee0     rtmp_init.obj
 0001:00003f10       ??_C@_1CG@JEBJJGB@?$AAA?$AAd?$AAh?$AAo?$AAc?$AAN?$AA4?$AA0?$AAM?$AAH?$AAz?$AAA?$AAl?$AAl?$AAo?$AAw?$AAe?$AAd?$AA?$AA@ 10004f10     rtmp_init.obj
 0001:00003f38       ??_C@_1BO@GPLOFEO@?$AAA?$AAd?$AAh?$AAo?$AAc?$AA5?$AAG?$AAD?$AAi?$AAs?$AAa?$AAb?$AAl?$AAe?$AA?$AA@ 10004f38     rtmp_init.obj
 0001:00003f58       ??_C@_1DC@PEAJAPLG@?$AAA?$AAd?$AAh?$AAo?$AAc?$AAN?$AAF?$AAo?$AAr?$AAc?$AAe?$AAM?$AAu?$AAl?$AAt?$AAi?$AAc?$AAa?$AAs?$AAt?$AAR?$AAa?$AAt?$AAe?$AA?$AA@ 10004f58     rtmp_init.obj
 0001:00003f8c       ??_C@_1BG@HIJECENL@?$AAA?$AAd?$AAh?$AAo?$AAc?$AAN?$AAM?$AAo?$AAd?$AAe?$AA?$AA@ 10004f8c     rtmp_init.obj
 0001:00003fa4       ??_C@_1BE@KABNOABI@?$AAA?$AAd?$AAh?$AAo?$AAc?$AAO?$AAf?$AAd?$AAm?$AA?$AA@ 10004fa4     rtmp_init.obj
 0001:00003fb8       ??_C@_1BI@FJLDDKCH@?$AAN?$AAe?$AAt?$AAw?$AAo?$AAr?$AAk?$AAT?$AAy?$AAp?$AAe?$AA?$AA@ 10004fb8     rtmp_init.obj
 0001:00003fd0       ??_C@_1BM@EFMHHLJG@?$AAA?$AAu?$AAt?$AAo?$AAR?$AAe?$AAc?$AAo?$AAn?$AAn?$AAe?$AAc?$AAt?$AA?$AA@ 10004fd0     rtmp_init.obj
 0001:00003fec       ??_C@_1BO@MJECKBG@?$AAS?$AAh?$AAo?$AAw?$AAH?$AAi?$AAd?$AAd?$AAe?$AAn?$AAS?$AAS?$AAI?$AAD?$AA?$AA@ 10004fec     rtmp_init.obj
 0001:0000400c       ??_C@_1M@HCFAIFML@?$AAR?$AAa?$AAd?$AAi?$AAo?$AA?$AA@ 1000500c     rtmp_init.obj
 0001:00004018       ??_C@_1BC@CKIBMGHF@?$AAP?$AAS?$AAP?$AAX?$AAl?$AAi?$AAn?$AAk?$AA?$AA@ 10005018     rtmp_init.obj
 0001:0000402c       ??_C@_1BG@LDMHCIGI@?$AAD?$AAi?$AAr?$AAe?$AAc?$AAt?$AAM?$AAo?$AAd?$AAe?$AA?$AA@ 1000502c     rtmp_init.obj
 0001:00004044       ??_C@_1BG@LEFEDPAE@?$AAD?$AAL?$AAS?$AAC?$AAa?$AAp?$AAa?$AAb?$AAl?$AAe?$AA?$AA@ 10005044     rtmp_init.obj
 0001:0000405c       ??_C@_1CA@EFEMNLAK@?$AAT?$AAr?$AAa?$AAn?$AAs?$AAm?$AAi?$AAt?$AAS?$AAe?$AAt?$AAt?$AAi?$AAn?$AAg?$AA?$AA@ 1000505c     rtmp_init.obj
 0001:0000407c       ??_C@_1BK@JLNNNNCD@?$AAB?$AAA?$AAC?$AAa?$AAp?$AAa?$AAb?$AAi?$AAl?$AAi?$AAt?$AAy?$AA?$AA@ 1000507c     rtmp_init.obj
 0001:00004098       ??_C@_1BI@HGMLCLKI@?$AAM?$AAu?$AAl?$AAt?$AAi?$AAp?$AAl?$AAe?$AAI?$AAR?$AAP?$AA?$AA@ 10005098     rtmp_init.obj
 0001:000040b0       ??_C@_1BI@FBEBBJAC@?$AAM?$AAa?$AAx?$AAS?$AAP?$AAL?$AAe?$AAn?$AAg?$AAt?$AAh?$AA?$AA@ 100050b0     rtmp_init.obj
 0001:000040c8       ??_C@_1BE@MGPCNCPB@?$AAA?$AAP?$AAS?$AAD?$AAA?$AAC?$AA_?$AAV?$AAO?$AA?$AA@ 100050c8     rtmp_init.obj
 0001:000040dc       ??_C@_1BE@ODJJINCN@?$AAA?$AAP?$AAS?$AAD?$AAA?$AAC?$AA_?$AAV?$AAI?$AA?$AA@ 100050dc     rtmp_init.obj
 0001:000040f0       ??_C@_1BE@NBNHAFCL@?$AAA?$AAP?$AAS?$AAD?$AAA?$AAC?$AA_?$AAB?$AAK?$AA?$AA@ 100050f0     rtmp_init.obj
 0001:00004104       ??_C@_1BE@DBAIHCBI@?$AAA?$AAP?$AAS?$AAD?$AAA?$AAC?$AA_?$AAB?$AAE?$AA?$AA@ 10005104     rtmp_init.obj
 0001:00004118       ??_C@_1BI@LOMHIPGP@?$AAA?$AAP?$AAS?$AAD?$AAC?$AAa?$AAp?$AAa?$AAb?$AAl?$AAe?$AA?$AA@ 10005118     rtmp_init.obj
 0001:00004130       ??_C@_1BG@HGDCKNNC@?$AAW?$AAM?$AAM?$AAC?$AAa?$AAp?$AAa?$AAb?$AAl?$AAe?$AA?$AA@ 10005130     rtmp_init.obj
 0001:00004148       ??_C@_1BI@OECFHPPP@?$AAT?$AAG?$AAn?$AAW?$AAi?$AAf?$AAi?$AAT?$AAe?$AAs?$AAt?$AA?$AA@ 10005148     rtmp_init.obj
 0001:00004160       ??_C@_1BA@FANIFMBI@?$AAT?$AAX?$AAB?$AAu?$AAr?$AAs?$AAt?$AA?$AA@ 10005160     rtmp_init.obj
 0001:00004170       ??_C@_1BM@GOCPLMJI@?$AAC?$AAa?$AAr?$AAr?$AAi?$AAe?$AAr?$AAD?$AAe?$AAt?$AAe?$AAc?$AAt?$AA?$AA@ 10005170     rtmp_init.obj
 0001:0000418c       ??_C@_1BG@BPJAKMMA@?$AAI?$AAE?$AAE?$AAE?$AA8?$AA0?$AA2?$AA1?$AA1?$AAH?$AA?$AA@ 1000518c     rtmp_init.obj
 0001:000041a4       ??_C@_1CC@CENNGNJ@?$AAF?$AAr?$AAa?$AAm?$AAe?$AAA?$AAg?$AAg?$AAr?$AAe?$AAg?$AAa?$AAt?$AAi?$AAo?$AAn?$AA?$AA@ 100051a4     rtmp_init.obj
 0001:000041c8       ??_C@_1BE@CJFJGBPC@?$AAS?$AAh?$AAo?$AAr?$AAt?$AAS?$AAl?$AAo?$AAt?$AA?$AA@ 100051c8     rtmp_init.obj
 0001:000041dc       ??_C@_1BK@KPPOILKG@?$AAB?$AAG?$AAP?$AAr?$AAo?$AAt?$AAe?$AAc?$AAt?$AAi?$AAo?$AAn?$AA?$AA@ 100051dc     rtmp_init.obj
 0001:000041f8       ??_C@_1CA@PGBNFBEB@?$AAM?$AAa?$AAx?$AAP?$AAk?$AAt?$AAO?$AAn?$AAe?$AAT?$AAx?$AAB?$AAu?$AAl?$AAk?$AA?$AA@ 100051f8     rtmp_init.obj
 0001:00004218       ??_C@_1BC@IOGOHBPE@?$AAT?$AAB?$AAF?$AAa?$AAc?$AAt?$AAo?$AAr?$AA?$AA@ 10005218     rtmp_init.obj
 0001:0000422c       ??_C@_1BC@IABCMNHB@?$AAR?$AAB?$AAF?$AAa?$AAc?$AAt?$AAo?$AAr?$AA?$AA@ 1000522c     rtmp_init.obj
 0001:00004240       ??_C@_1BO@HGPPFMIN@?$AAN?$AAe?$AAt?$AAw?$AAo?$AAr?$AAk?$AAA?$AAd?$AAd?$AAr?$AAe?$AAs?$AAs?$AA?$AA@ 10005240     rtmp_init.obj
 0001:00004260       ??_C@_1BA@HCLACGFM@?$AAW?$AAE?$AAP?$AAK?$AAe?$AAy?$AA4?$AA?$AA@ 10005260     rtmp_init.obj
 0001:00004270       ??_C@_1BA@OPGHBOOF@?$AAW?$AAE?$AAP?$AAK?$AAe?$AAy?$AA3?$AA?$AA@ 10005270     rtmp_init.obj
 0001:00004280       ??_C@_1BA@FHNLHJIA@?$AAW?$AAE?$AAP?$AAK?$AAe?$AAy?$AA2?$AA?$AA@ 10005280     rtmp_init.obj
 0001:00004290       ??_C@_1BA@EFGONGGO@?$AAW?$AAE?$AAP?$AAK?$AAe?$AAy?$AA1?$AA?$AA@ 10005290     rtmp_init.obj
 0001:000042a0       ??_C@_1BG@OHMGBAFO@?$AAW?$AAP?$AAS?$AAD?$AAe?$AAv?$AAN?$AAa?$AAm?$AAe?$AA?$AA@ 100052a0     rtmp_init.obj
 0001:000042b8       ??_C@_1BG@OIMBEMPB@?$AAV?$AAe?$AAn?$AAd?$AAo?$AAr?$AAD?$AAe?$AAs?$AAc?$AA?$AA@ 100052b8     rtmp_init.obj
 0001:000042d0       ??_C@_19KJNOMKCJ@?$AAS?$AAS?$AAI?$AAD?$AA?$AA@ 100052d0     rtmp_init.obj
 0001:000042dc       ??_C@_17BPNEPMND@?$AAR?$AAD?$AAG?$AA?$AA@ 100052dc     rtmp_init.obj
 0001:000042e4       ??_C@_1BE@HKNKOMJL@?$AAW?$AAE?$AAP?$AAK?$AAe?$AAy?$AAU?$AAs?$AAe?$AA?$AA@ 100052e4     rtmp_init.obj
 0001:000042f8       ??_C@_1BG@CLENCLJC@?$AAA?$AAu?$AAt?$AAh?$AAe?$AAn?$AAT?$AAy?$AAp?$AAe?$AA?$AA@ 100052f8     rtmp_init.obj
 0001:00004310       ??_C@_1BG@MHEIMMBG@?$AAE?$AAn?$AAc?$AAr?$AAy?$AAp?$AAt?$AAi?$AAo?$AAn?$AA?$AA@ 10005310     rtmp_init.obj
 0001:00004328       ??_C@_1BG@CPCOBECG@?$AAF?$AAr?$AAa?$AAg?$AAT?$AAh?$AAr?$AAe?$AAs?$AAh?$AA?$AA@ 10005328     rtmp_init.obj
 0001:00004340       ??_C@_1BE@NCNOFIOB@?$AAR?$AAt?$AAs?$AAT?$AAh?$AAr?$AAe?$AAs?$AAh?$AA?$AA@ 10005340     rtmp_init.obj
 0001:00004354       ??_C@_1BA@DLAHBHMC@?$AAC?$AAh?$AAa?$AAn?$AAn?$AAe?$AAl?$AA?$AA@ 10005354     rtmp_init.obj
 0001:00004364       ??_C@_1BK@CMGABJAK@?$AAW?$AAi?$AAr?$AAe?$AAl?$AAe?$AAs?$AAs?$AAM?$AAo?$AAd?$AAe?$AA?$AA@ 10005364     rtmp_init.obj
 0001:00004380       ??_C@_1CG@FHJPKHBD@?$AAC?$AAo?$AAu?$AAn?$AAt?$AAr?$AAy?$AAR?$AAe?$AAg?$AAi?$AAo?$AAn?$AAA?$AAB?$AAa?$AAn?$AAd?$AA?$AA@ 10005380     rtmp_init.obj
 0001:000043a8       ??_C@_1BM@PHDEHLBE@?$AAC?$AAo?$AAu?$AAn?$AAt?$AAr?$AAy?$AAR?$AAe?$AAg?$AAi?$AAo?$AAn?$AA?$AA@ 100053a8     rtmp_init.obj
 0001:000043c4       ??_C@_1CA@PGOEGKAH@?$AAU?$AAs?$AAe?$AAR?$AAa?$AAS?$AAu?$AAp?$AAp?$AAl?$AAi?$AAc?$AAa?$AAn?$AAt?$AA?$AA@ 100053c4     rtmp_init.obj
 0001:000043e4       ??_C@_1O@OADBDALB@?$AAO?$AAp?$AAM?$AAo?$AAd?$AAe?$AA?$AA@ 100053e4     rtmp_init.obj
 0001:000043f4       ??_C@_07BDGAECLF@CKIP128?$AA@ 100053f4     rtmp_init.obj
 0001:000043fc       ??_C@_07LMFBNJNH@CKIP104?$AA@ 100053fc     rtmp_init.obj
 0001:00004404       ??_C@_06HHMNOKIF@CKIP64?$AA@ 10005404     rtmp_init.obj
 0001:0000440c       ??_C@_03BKNEFOAH@AES?$AA@  1000540c     rtmp_init.obj
 0001:00004410       ??_C@_04HNKLFFMO@TKIP?$AA@ 10005410     rtmp_init.obj
 0001:00004418       ??_C@_06JCFAKCMD@wep128?$AA@ 10005418     rtmp_init.obj
 0001:00004420       ??_C@_05PJDLFBFB@wep64?$AA@ 10005420     rtmp_init.obj
 0001:00004428       ??_C@_04CGFJFPFD@none?$AA@ 10005428     rtmp_init.obj
 0001:00004630       ccitt_16Table              10005630     rtmp_init.obj
 0001:00004830       ??_C@_1BM@IBPGOOAH@?$AAC?$AAo?$AAn?$AAt?$AAr?$AAo?$AAl?$AA?5?$AAE?$AAv?$AAe?$AAn?$AAt?$AA?$AA@ 10005830     rtmp_init.obj
 0001:0000484c       ??_C@_1BG@EEMGAPFL@?$AAM?$AAL?$AAM?$AAE?$AA?5?$AAE?$AAv?$AAe?$AAn?$AAt?$AA?$AA@ 1000584c     rtmp_init.obj
 0001:00004864       ??_C@_1BG@KDOEMPEF@?$AAJ?$AAu?$AAn?$AAk?$AA?5?$AAE?$AAv?$AAe?$AAn?$AAt?$AA?$AA@ 10005864     rtmp_init.obj
 0001:0000487c       ??_C@_1CA@EGHOFHML@?$AAS?$AAa?$AAf?$AAe?$AAl?$AAy?$AAR?$AAe?$AAm?$AAo?$AAv?$AAe?$AAO?$AAf?$AAf?$AA?$AA@ 1000587c     rtmp_init.obj
 0001:0000489c       ??_C@_0L@KBGDKEEF@rt2870?4bin?$AA@ 1000589c     rtmp_init.obj
 0001:000050a8       ??_C@_1LM@NKJIMFHB@?$AAR?$AAT?$AA2?$AA8?$AA7?$AA0?$AA?3?$AA?5?$AA?$CK?$AA?$CK?$AA?$CK?$AAD?$AAu?$AAm?$AAp?$AA?3?$AA?5?$AAB?$AAe?$AAf?$AAo?$AAr?$AAe?$AA?3?$AA?5?$AAR?$AAT?$AAU?$AAS?$AAB?$AAE?$AAn@ 100060a8     rtusb_bulk.obj
 0001:00005168       ??_C@_1LM@DGIIDKDA@?$AAR?$AAT?$AA2?$AA8?$AA7?$AA0?$AA?3?$AA?5?$AA?$CK?$AA?$CK?$AA?$CK?$AAD?$AAu?$AAm?$AAp?$AA?3?$AA?5?$AAA?$AAf?$AAt?$AAe?$AAr?$AA?5?$AA?3?$AA?5?$AAR?$AAT?$AAU?$AAS?$AAB?$AAE?$AAn@ 10006168     rtusb_bulk.obj
 0001:00005224       ??_C@_02JJDEPCGB@54?$AA@   10006224     rtusb_data.obj
 0001:00005228       ??_C@_02DEEDNHFK@48?$AA@   10006228     rtusb_data.obj
 0001:0000522c       ??_C@_02KPIPOMFB@36?$AA@   1000622c     rtusb_data.obj
 0001:00005230       ??_C@_02JMHLOEOE@24?$AA@   10006230     rtusb_data.obj
 0001:00005234       ??_C@_02DCIIBFLB@18?$AA@   10006234     rtusb_data.obj
 0001:00005238       ??_C@_02MIGHPNDL@12?$AA@   10006238     rtusb_data.obj
 0001:0000523c       ??_C@_01LAKCGALK@9?$AA@    1000623c     rtusb_data.obj
 0001:00005240       ??_C@_01DHDKHMHF@6?$AA@    10006240     rtusb_data.obj
 0001:00005448       ??_C@_08DLGAODGK@BYE?5sip?3?$AA@ 10006448     rtusb_data.obj
 0001:00005454       ??_C@_0M@NPADNAGD@CANCEL?5sip?3?$AA@ 10006454     rtusb_data.obj
 0001:00005460       ??_C@_0M@CCBCPDCA@INVITE?5sip?3?$AA@ 10006460     rtusb_data.obj
 0001:00005e70       ??_C@_1BA@CCMJLFHB@?$AAR?$AAT?$AA2?$AA8?$AA7?$AA0?$AA1?$AA?$AA@ 10006e70     wince.obj
 0001:00005e80       ??_C@_1O@ECGDNAC@?$AAR?$AAT?$AA2?$AA8?$AA7?$AA0?$AA?$AA@ 10006e80     wince.obj
 0001:00005e90       ??_C@_1BM@OOGBHLFH@?$AAC?$AAu?$AAs?$AAt?$AAo?$AAm?$AAi?$AAz?$AAe?$AAd?$AAP?$AAI?$AAD?$AA?$AA@ 10006e90     wince.obj
 0001:00005eac       ??_C@_1BM@CIAOHCNA@?$AAC?$AAu?$AAs?$AAt?$AAo?$AAm?$AAi?$AAz?$AAe?$AAd?$AAV?$AAI?$AAD?$AA?$AA@ 10006eac     wince.obj
 0001:00005ec8       ??_C@_1CM@CEPJCBLC@?$AAC?$AAu?$AAs?$AAt?$AAo?$AAm?$AAi?$AAz?$AAe?$AAd?$AAC?$AAo?$AAn?$AAt?$AAr?$AAo?$AAl?$AAF?$AAl?$AAa?$AAg?$AA?$AA@ 10006ec8     wince.obj
 0001:00005ef4       ??_C@_1CG@GEIBFOOG@?$AAC?$AAo?$AAm?$AAm?$AA?2?$AAR?$AAT?$AA2?$AA8?$AA7?$AA0?$AA1?$AA?2?$AAP?$AAa?$AAr?$AAm?$AAs?$AA?$AA@ 10006ef4     wince.obj
 0001:00005f20       ??_C@_1GK@EFNNGGDG@?$AAD?$AAe?$AAv?$AAi?$AAc?$AAe?$AA?5?$AAi?$AAs?$AA?5?$AAn?$AAo?$AAt?$AA?5?$AAm?$AAa?$AAt?$AAc?$AAh?$AAe?$AAd?$AA?5?$AAc?$AAu?$AAs?$AAt?$AAo?$AAm?$AAe?$AAr?$AA?8?$AAs@ 10006f20     wince.obj
 0001:00005f90       ??_C@_1HM@IGPJLFMJ@?$AAT?$AAh?$AAi?$AAs?$AA?5?$AAd?$AAe?$AAv?$AAi?$AAc?$AAe?$AA?5?$AAi?$AAs?$AA?5?$AAn?$AAo?$AAt?$AA?5?$AAf?$AAo?$AAu?$AAn?$AAd?$AA?5?$AAi?$AAn?$AA?5?$AAt?$AAh?$AAe?$AA?5@ 10006f90     wince.obj
 0001:0000600c       ??_C@_1DM@GIKJLEAJ@?$AAD?$AAe?$AAv?$AAi?$AAc?$AAe?$AA?$CI?$AAV?$AAI?$AAD?$AA?$DN?$AA0?$AAx?$AA?$CF?$AA0?$AA4?$AAx?$AA?0?$AA?5?$AAP?$AAI?$AAD?$AA?$DN?$AA0?$AAx?$AA?$CF?$AA4?$AAx?$AA?$CJ?$AA?$AA@ 1000700c     wince.obj
 0001:00006048       ??_C@_1BM@KHHDMGEP@?$AAP?$AAa?$AAg?$AAe?$AAS?$AAi?$AAz?$AAe?$AA?$DN?$AA?$CF?$AAd?$AA?$AN?$AA?6?$AA?$AA@ 10007048     wince.obj
 0001:00006064       ??_C@_1CI@BKHJAAEJ@?$AAP?$AAr?$AAo?$AAc?$AAe?$AAs?$AAs?$AAo?$AAr?$AAL?$AAe?$AAv?$AAe?$AAl?$AA?$DN?$AA?$CF?$AAd?$AA?$AN?$AA?6?$AA?$AA@ 10007064     wince.obj
 0001:0000608c       ??_C@_1DC@LKOADMHA@?$AAP?$AAr?$AAo?$AAc?$AAe?$AAs?$AAs?$AAo?$AAr?$AAR?$AAe?$AAv?$AAi?$AAs?$AAi?$AAo?$AAn?$AA?$DN?$AA?$CF?$AA0?$AA4?$AAx?$AA?$AN?$AA?6?$AA?$AA@ 1000708c     wince.obj
 0001:000060c0       ??_C@_1BI@MPBJOOFH@?$AAC?$AAP?$AAU?$AA?$DN?$AAI?$AAn?$AAt?$AAe?$AAl?$AA?$AN?$AA?6?$AA?$AA@ 100070c0     wince.obj
 0001:000060d8       ??_C@_1BI@LDGJLFJC@?$AAC?$AAP?$AAU?$AA?$DN?$AAM?$AAI?$AAP?$AAS?$AA?5?$AA?$AN?$AA?6?$AA?$AA@ 100070d8     wince.obj
 0001:000060f0       ??_C@_1BE@EEFFOFNO@?$AAC?$AAP?$AAU?$AA?$DN?$AAS?$AAH?$AA4?$AA?$AN?$AA?6?$AA?$AA@ 100070f0     wince.obj
 0001:00006104       ??_C@_1BE@CHOFANCH@?$AAC?$AAP?$AAU?$AA?$DN?$AAA?$AAR?$AAM?$AA?$AN?$AA?6?$AA?$AA@ 10007104     wince.obj
 0001:00006118       ??_C@_1BM@EJAINDLO@?$AAC?$AAP?$AAU?$AA?$DN?$AAU?$AAN?$AAK?$AAN?$AAO?$AAW?$AAN?$AA?$AN?$AA?6?$AA?$AA@ 10007118     wince.obj
 0001:00006134       ??_C@_1CM@BHHLIDEJ@?$AAR?$AAT?$AA2?$AA8?$AA7?$AA0?$AA?3?$AA?$DM?$AA?$DN?$AA?$DN?$AA?5?$AAD?$AAl?$AAl?$AAE?$AAn?$AAt?$AAr?$AAy?$AA?$AN?$AA?6?$AA?$AA@ 10007134     wince.obj
 0001:00006160       ??_C@_1DK@HDOFPFHO@?$AAR?$AAT?$AA2?$AA8?$AA7?$AA0?$AA?3?$AA?5?$AAD?$AAL?$AAL?$AA_?$AAP?$AAR?$AAO?$AAC?$AAE?$AAS?$AAS?$AA_?$AAD?$AAE?$AAT?$AAA?$AAC?$AAH?$AA?$AN?$AA?6?$AA?$AA@ 10007160     wince.obj
 0001:0000619c       ??_C@_1DK@NPFADLJG@?$AAR?$AAT?$AA2?$AA8?$AA7?$AA0?$AA?3?$AA?5?$AAD?$AAL?$AAL?$AA_?$AAP?$AAR?$AAO?$AAC?$AAE?$AAS?$AAS?$AA_?$AAA?$AAT?$AAT?$AAA?$AAC?$AAH?$AA?$AN?$AA?6?$AA?$AA@ 1000719c     wince.obj
 0001:000061d8       ??_C@_1FC@COJHCDK@?$AAB?$AAu?$AAi?$AAl?$AAd?$AA?5?$AAD?$AAa?$AAt?$AAe?$AA?3?$AA?5?$AAD?$AAe?$AAc?$AA?5?$AA?5?$AA4?$AA?5?$AA2?$AA0?$AA0?$AA9?$AA?5?$AAT?$AAi?$AAm?$AAe?$AA?3?$AA?5?$AA1?$AA7@ 100071d8     wince.obj
 0001:0000622c       ??_C@_1DO@HNGPEDBJ@?$AAD?$AAr?$AAi?$AAv?$AAe?$AAr?$AA?5?$AAV?$AAe?$AAr?$AAs?$AAi?$AAo?$AAn?$AA?3?$AA?5?$AA0?$AAx?$AA?$CF?$AA0?$AA8?$AAx?$AA?5?$AA?$CI?$AAR?$AAE?$AAL?$AA?$CJ?$AA?$AN?$AA?6?$AA?$AA@ 1000722c     wince.obj
 0001:0000626c       ??_C@_1CM@NJEMINLJ@?$AAR?$AAT?$AA2?$AA8?$AA7?$AA0?$AA?3?$AA?$DN?$AA?$DN?$AA?$DO?$AA?5?$AAD?$AAl?$AAl?$AAE?$AAn?$AAt?$AAr?$AAy?$AA?$AN?$AA?6?$AA?$AA@ 1000726c     wince.obj
 0001:00006698       ??_C@_0IB@NJPMFJAK@?$CF02X?$CF02X?$CF02X?$CF02X?$CF02X?$CF02X?$CF02X?$CF02X@ 10007698     wsc.obj
 0001:0000671c       ??_C@_0BE@HGMAMNJC@ExRegNW?$CF02X?$CF02X?$CF02X?$AA@ 1000771c     wsc.obj
 0001:00006930       k256                       10007930     wsc_crypto.obj
 0001:00006a30       i256                       10007a30     wsc_crypto.obj
 0001:00009678       ??_C@_08PDCNPKJD@TDLS?5PMK?$AA@ 1000a678     tdls.obj
 0001:000096a8       MlmeQOSAction              1000a6a8 f   action.obj
 0001:000096ac       MlmeInvalidAction          1000a6ac f   action.obj
 0001:000096b0       PeerDelBAAction            1000a6b0 f   action.obj
 0001:000098fc       PeerQOSAction              1000a8fc f   action.obj
 0001:00009908       StaPeerPublicAction        1000a908 f   action.obj
 0001:000099d0       PeerRMAction               1000a9d0 f   action.obj
 0001:000099dc       PeerHTAction               1000a9dc f   action.obj
 0001:00009b48       RECBATimerTimeout          1000ab48 f   action.obj
 0001:00009f7c       ActHeaderInit              1000af7c f   action.obj
 0001:0000a0b4       BarHeaderInit              1000b0b4 f   action.obj
 0001:0000a1f4       QosBADataParse             1000b1f4 f   action.obj
 0001:0000b1ac       CntlEnqueueForRecv         1000c1ac f   action.obj
 0001:0000b8bc       BaAutoManSwitch            1000c8bc f   action.obj
 0001:0000ba10       SendPSMPAction             1000ca10 f   action.obj
 0001:0000bc9c       ChannelSwitchSanityCheck   1000cc9c f   action.obj
 0001:0000bd34       ChannelSwitchAction        1000cd34 f   action.obj
 0001:0000bfd0       BuildIntolerantChannelRep  1000cfd0 f   action.obj
 0001:0000c1c4       Send2040CoexistAction      1000d1c4 f   action.obj
 0001:0000c308       UpdateBssScanParm          1000d308 f   action.obj
 0001:0000c5c0       MlmeADDBAAction            1000d5c0 f   action.obj
 0001:0000c774       MlmeDELBAAction            1000d774 f   action.obj
 0001:0000c9ac       PeerAddBAReqAction         1000d9ac f   action.obj
 0001:0000ce88       PeerAddBARspAction         1000de88 f   action.obj
 0001:0000d354       PeerSpectrumAction         1000e354 f   action.obj
 0001:0000d40c       PeerBAAction               1000e40c f   action.obj
 0001:0000d450       PeerPublicAction           1000e450 f   action.obj
 0001:0000d4b4       ORIBATimerTimeout          1000e4b4 f   action.obj
 0001:0000db34       Update2040CoexistFrameAndNotify 1000eb34 f   action.obj
 0001:0000db64       ActionStateMachineInit     1000eb64 f   action.obj
 0001:0000dcb0       ACM_WME_ActionFrameBodyMake 1000ecb0 f   acm_action.obj
 0001:0000dd5c       AcmCmdAddTSRequest         1000ed5c f   acm_action.obj
 0001:0000ded8       AcmPeerRspHandle           1000eed8 f   acm_action.obj
 0001:0000e118       AcmCmdDelTSSend            1000f118 f   acm_action.obj
 0001:0000e230       AcmCmdTclasReset           1000f230 f   acm_action.obj
 0001:0000e270       AcmReqCmdAction            1000f270 f   acm_action.obj
 0001:0000e56c       AcmStateMachineInit        1000f56c f   acm_action.obj
 0001:0000e624       RTMPusecDelay              1000f624 f i aironet.obj
 0001:0000e674       ChannelLoadRequestAction   1000f674 f   aironet.obj
 0001:0000e7a0       NoiseHistRequestAction     1000f7a0 f   aironet.obj
 0001:0000e8f8       FrameRequestAction         1000f8f8 f   aironet.obj
 0001:0000ea38       StatisticsRequestAction    1000fa38 f   aironet.obj
 0001:0000eb20       ChannelLoadReportAction    1000fb20 f   aironet.obj
 0001:0000edb4       NoiseHistReportAction      1000fdb4 f   aironet.obj
 0001:0000f2bc       AironetAddBeaconReport     100102bc f   aironet.obj
 0001:0000f678       AironetCreateBeaconReportFromBssTable 10010678 f   aironet.obj
 0001:0000f998       AironetAddFrameTestReport  10010998 f   aironet.obj
 0001:0000fba8       FrameTestReportAction      10010ba8 f   aironet.obj
 0001:0000fcec       PathLossTimeOutAction      10010cec f   aironet.obj
 0001:0000fd98       PathLossMessageAction      10010d98 f   aironet.obj
 0001:00010094       StatisticsReportAction     10011094 f   aironet.obj
 0001:000105d4       CCXAironetTimeOutAction    100115d4 f   aironet.obj
 0001:00010610       AironetDirectRoam          10011610 f   aironet.obj
 0001:00010824       CCXSearchNBLToSwap         10011824 f   aironet.obj
 0001:000108c8       ConvertRssiToSignalQuality 100118c8 f   aironet.obj
 0001:0001090c       SendAironetReport          1001190c f   aironet.obj
 0001:00010a8c       InitCACTspec               10011a8c f   aironet.obj
 0001:00010d14       CacTsMetricsRptTimeoutAction 10011d14 f   aironet.obj
 0001:00011030       AironetApLogTableInit      10012030 f   aironet.obj
 0001:00011060       AironetApLogEntryUpdate    10012060 f   aironet.obj
 0001:000110d0       AironetApLogEntrySet       100120d0 f   aironet.obj
 0001:0001114c       AironetApLogTableSetNewEntry 1001214c f   aironet.obj
 0001:00011318       SendEAPOLStart             10012318 f   aironet.obj
 0001:00011530       AironetRFRoaming           10012530 f   aironet.obj
 0001:000116ec       AironetASTScanReq          100126ec f   aironet.obj
 0001:00011814       CCXDiagInitMemoryHandler   10012814 f   aironet.obj
 0001:0001191c       CCXDiagGetMemory           1001291c f   aironet.obj
 0001:000119e8       CCXDiagFreeMemoryHandler   100129e8 f   aironet.obj
 0001:00011a68       CCXDiagLogFrame            10012a68 f   aironet.obj
 0001:00011ac0       TxCCXDiagLogFrames         10012ac0 f   aironet.obj
 0001:00011d38       BeaconRequestAction        10012d38 f   aironet.obj
 0001:00011f04       AironetLogRequestAction    10012f04 f   aironet.obj
 0001:000123c0       AironetFinalReportAction   100133c0 f   aironet.obj
 0001:00012668       PathLossReportAction       10013668 f   aironet.obj
 0001:0001292c       AironetL2RoamingAction     1001392c f   aironet.obj
 0001:00012a3c       AironetLinkTestAction      10013a3c f   aironet.obj
 0001:00012e34       TxAironetFromSupplicantAction 10013e34 f   aironet.obj
 0001:00012f7c       AironetMsgAction           10013f7c f   aironet.obj
 0001:000133bc       PathLossRequestAction      100143bc f   aironet.obj
 0001:000135fc       AironetReportAction        100145fc f   aironet.obj
 0001:00013794       AironetRequestAction       10014794 f   aironet.obj
 0001:000138d0       AironetStateMachineInit    100148d0 f   aironet.obj
 0001:000139ec       APInitialize               100149ec f   ap.obj
 0001:00013a74       APCleanupPsQueue           10014a74 f   ap.obj
 0001:00013b1c       ApLogEvent                 10014b1c f   ap.obj
 0001:00013bc0       APUpdateOperationMode      10014bc0 f   ap.obj
 0001:00013cac       APUpdateCapabilityAndErpIe 10014cac f   ap.obj
 0001:00013ecc       ApCheckAccessControlList   10014ecc f   ap.obj
 0001:00013f6c       APPsIndicate               10014f6c f   ap.obj
 0001:00014020       MacTableInitialize         10015020 f   ap.obj
 0001:000140f4       MacTableReset              100150f4 f   ap.obj
 0001:0001436c       MacTableInsertEntry        1001536c f   ap.obj
 0001:00014628       MacTableDeleteEntry        10015628 f   ap.obj
 0001:000148e4       MacTableLookup             100158e4 f   ap.obj
 0001:000149b0       MacTableMaintenance        100159b0 f   ap.obj
 0001:00014cd0       WdsTableInsertEntry        10015cd0 f   ap.obj
 0001:00014e7c       WdsTableDeleteEntry        10015e7c f   ap.obj
 0001:00014fcc       WdsTableLookup             10015fcc f   ap.obj
 0001:00015080       ApUpdateAccessControlList  10016080 f   ap.obj
 0001:00015344       APStartUp                  10016344 f   ap.obj
 0001:00015e5c       APStop                     10016e5c f   ap.obj
 0001:00015f54       APShutdown                 10016f54 f   ap.obj
 0001:00015fe4       APSsPsInquiry              10016fe4 f   ap.obj
 0001:000160a0       APPeerDisassocReqAction    100170a0 f   ap_assoc.obj
 0001:00016124       APMlmeDisassocReqAction    10017124 f   ap_assoc.obj
 0001:0001620c       APCls3errAction            1001720c f   ap_assoc.obj
 0001:000162e8       APBuildAssociation         100172e8 f   ap_assoc.obj
 0001:00016bf8       APPeerAssocReqAction       10017bf8 f   ap_assoc.obj
 0001:000173a4       APPeerReassocReqAction     100183a4 f   ap_assoc.obj
 0001:00017b50       APAssocStateMachineInit    10018b50 f   ap_assoc.obj
 0001:00017c00       APMlmeDeauthReqAction      10018c00 f   ap_auth.obj
 0001:00017ce8       APCls2errAction            10018ce8 f   ap_auth.obj
 0001:00017dc4       APAuthStateMachineInit     10018dc4 f   ap_auth.obj
 0001:00017e2c       APPeerDeauthReqAction      10018e2c f   ap_authrsp.obj
 0001:00017f00       APPeerAuthSimpleRspGenAndSend 10018f00 f   ap_authrsp.obj
 0001:00018044       APPeerAuthAtAuthRspIdleAction 10019044 f   ap_authrsp.obj
 0001:00018544       APAuthRspStateMachineInit  10019544 f   ap_authrsp.obj
 0001:000185dc       APMakeBssBeacon            100195dc f   ap_connect.obj
 0001:00018bf4       APUpdateBeaconFrame        10019bf4 f   ap_connect.obj
 0001:0001932c       APSendPacket               1001a32c f   ap_data.obj
 0001:000196e4       APHardTransmit             1001a6e4 f   ap_data.obj
 0001:0001b234       APCheckClass2Class3Error   1001c234 f   ap_data.obj
 0001:0001b2a0       APHandleRxPsPoll           1001c2a0 f   ap_data.obj
 0001:0001b478       APBridgeToWdsAndWirelessSta 1001c478 f   ap_data.obj
 0001:0001b6cc       APCheckNDSClient           1001c6cc f   ap_data.obj
 0001:0001b7c4       APSendPackets              1001c7c4 f   ap_data.obj
 0001:0001ba00       RTUSBAPHandleRxPacket      1001ca00 f   ap_data.obj
 0001:0001d11c       APSetInformation           1001e11c f   ap_info.obj
 0001:0001df7c       APQueryInformation         1001ef7c f   ap_info.obj
 0001:0001e564       APMlmePeriodicExec         1001f564 f   ap_mlme.obj
 0001:0001e744       APMlmeSelectTxRateTable    1001f744 f   ap_mlme.obj
 0001:0001ead8       APMlmeSetTxRate            1001fad8 f   ap_mlme.obj
 0001:0001ec14       APMlmeDynamicTxRateSwitching 1001fc14 f   ap_mlme.obj
 0001:0001f6b4       APQuickResponeForRateUpExec 100206b4 f   ap_mlme.obj
 0001:0001fb30       APMsgTypeSubst             10020b30 f   ap_mlme.obj
 0001:0001fc90       RTMPSetPiggyBack           10020c90 f   ap_mlme.obj
 0001:0001fcdc       APAsicEvaluateRxAnt        10020cdc f   ap_mlme.obj
 0001:0001fda0       APAsicRxAntEvalTimeout     10020da0 f   ap_mlme.obj
 0001:0001fe7c       PeerAssocReqSanity         10020e7c f   ap_sanity.obj
 0001:000203d4       PeerReassocReqSanity       100213d4 f   ap_sanity.obj
 0001:000208d0       PeerDisassocReqSanity      100218d0 f   ap_sanity.obj
 0001:00020944       PeerDeauthReqSanity        10021944 f   ap_sanity.obj
 0001:000209b8       APPeerAuthSanity           100219b8 f   ap_sanity.obj
 0001:00020ac4       APPeerProbeReqSanity       10021ac4 f   ap_sanity.obj
 0001:00020b68       APPeerBeaconAndProbeRspSanity 10021b68 f   ap_sanity.obj
 0001:00020e68       APPeerProbeReqAction       10021e68 f   ap_sync.obj
 0001:00021764       APPeerBeaconAction         10022764 f   ap_sync.obj
 0001:000218f4       APSyncStateMachineInit     100228f4 f   ap_sync.obj
 0001:00021974       APWapiWAIPacket_HandleMBcastRsp 10022974 f   Ap_wapi.obj
 0001:00021c64       APSTAWapiGen_MIC           10022c64 f   Ap_wapi.obj
 0001:00021c9c       APSTAWapiGen_MBcastKey     10022c9c f   Ap_wapi.obj
 0001:00021cdc       APSTAWapiGen_BKAndChallengeSeed 10022cdc f   Ap_wapi.obj
 0001:00021d64       APSTAWapiGen_BKID          10022d64 f   Ap_wapi.obj
 0001:00021da4       APSTAWapiGen_PairwiseKey   10022da4 f   Ap_wapi.obj
 0001:00021e4c       SMS4Crypt                  10022e4c f   Ap_wapi.obj
 0001:000220ac       SMS4KeyExt                 100230ac f   Ap_wapi.obj
 0001:000222b8       wpi_encrypt                100232b8 f   Ap_wapi.obj
 0001:000223ac       wpi_decrypt                100233ac f   Ap_wapi.obj
 0001:000223cc       wpi_pmac                   100233cc f   Ap_wapi.obj
 0001:000224b0       APSTA_IV_ADD               100234b0 f   Ap_wapi.obj
 0001:00022508       APSTA_IV_GREATER_THAN      10023508 f   Ap_wapi.obj
 0001:00022558       APWapiSend_MBcastKeyNegotiate_Req 10023558 f   Ap_wapi.obj
 0001:000228e8       APWapiSend_UnicastKeyNegotiate_Req 100238e8 f   Ap_wapi.obj
 0001:00022b9c       APWapiSend_UnicastKeyNegotiate_Conf 10023b9c f   Ap_wapi.obj
 0001:00022e1c       APWapiWAI_UnicastReq_Action 10023e1c f   Ap_wapi.obj
 0001:00022ef0       APWapiWAI_MBcastReq_Action 10023ef0 f   Ap_wapi.obj
 0001:00022f5c       APWapiWAIPacket_HandleUnicastRsp 10023f5c f   Ap_wapi.obj
 0001:000231ac       APWapiWAIPacketAction      100241ac f   Ap_wapi.obj
 0001:0002326c       APWapiStateMachineInit     1002426c f   Ap_wapi.obj
 0001:000232fc       WPAMsgTypeSubst            100242fc f   ap_wpa.obj
 0001:00023358       APWpaEAPPacketAction       10024358 f   ap_wpa.obj
 0001:0002335c       APWpaEAPOLASFAlertAction   1002435c f   ap_wpa.obj
 0001:00023360       APWpaEAPOLLogoffAction     10024360 f   ap_wpa.obj
 0001:00023364       PACInquiry                 10024364 f   ap_wpa.obj
 0001:00023388       RTMPCheckWPAframe          10024388 f   ap_wpa.obj
 0001:00023410       RTMPCheckMcast             10024410 f   ap_wpa.obj
 0001:000234fc       RTMPCheckUcast             100244fc f   ap_wpa.obj
 0001:00023634       RTMPCheckAUTH              10024634 f   ap_wpa.obj
 0001:0002373c       CMTimerExec                1002473c f   ap_wpa.obj
 0001:000237a4       Wpa2PeerPairMsg4Action     100247a4 f   ap_wpa.obj
 0001:000239ec       PeerGroupMsg2Action        100249ec f   ap_wpa.obj
 0001:00023b78       DisAssocAction             10024b78 f   ap_wpa.obj
 0001:00023c54       CountGTK                   10024c54 f   ap_wpa.obj
 0001:00023d8c       GetSmall                   10024d8c f   ap_wpa.obj
 0001:00023df4       GetLarge                   10024df4 f   ap_wpa.obj
 0001:00023e64       APGenRandom                10024e64 f   ap_wpa.obj
 0001:00024028       AES_GTK_KEY_WRAP           10025028 f   ap_wpa.obj
 0001:00024184       RTMPMakeRSNIE              10025184 f   ap_wpa.obj
 0001:00024738       APToWirelessSta            10025738 f   ap_wpa.obj
 0001:000248ec       HandleCounterMeasure       100258ec f   ap_wpa.obj
 0001:00024a28       WPAStart4WayHS             10025a28 f   ap_wpa.obj
 0001:00024bf4       WPAHardTransmit            10025bf4 f   ap_wpa.obj
 0001:000254d8       GREKEYPeriodicExec         100264d8 f   ap_wpa.obj
 0001:0002567c       CountPTK                   1002667c f   ap_wpa.obj
 0001:00025840       APWpaEAPOLStartAction      10026840 f   ap_wpa.obj
 0001:00025914       PeerPairMsg2Action         10026914 f   ap_wpa.obj
 0001:000261dc       WPARetryExec               100271dc f   ap_wpa.obj
 0001:0002647c       Wpa1PeerPairMsg4Action     1002747c f   ap_wpa.obj
 0001:000266cc       APWpaEAPOLKeyAction        100276cc f   ap_wpa.obj
 0001:00026988       APWpaStateMachineInit      10027988 f   ap_wpa.obj
 0001:00026a48       AssocTimeout               10027a48 f   assoc.obj
 0001:00026aa4       ReassocTimeout             10027aa4 f   assoc.obj
 0001:00026b00       DisassocTimeout            10027b00 f   assoc.obj
 0001:00026b64       MlmeAssocReqAction         10027b64 f   assoc.obj
 0001:000280ac       MlmeReassocReqAction       100290ac f   assoc.obj
 0001:00029130       MlmeDisassocReqAction      1002a130 f   assoc.obj
 0001:0002939c       AssocPostProc              1002a39c f   assoc.obj
 0001:00029628       PeerDisassocAction         1002a628 f   assoc.obj
 0001:00029824       AssocTimeoutAction         1002a824 f   assoc.obj
 0001:00029864       ReassocTimeoutAction       1002a864 f   assoc.obj
 0001:000298a4       DisassocTimeoutAction      1002a8a4 f   assoc.obj
 0001:000298e4       InvalidStateWhenAssoc      1002a8e4 f   assoc.obj
 0001:00029924       InvalidStateWhenReassoc    1002a924 f   assoc.obj
 0001:00029964       InvalidStateWhenDisassociate 1002a964 f   assoc.obj
 0001:000299ac       Cls3errAction              1002a9ac f   assoc.obj
 0001:00029b4c       SwitchBetweenWepAndCkip    1002ab4c f   assoc.obj
 0001:00029de4       PeerAssocRspAction         1002ade4 f   assoc.obj
 0001:0002a1f0       PeerReassocRspAction       1002b1f0 f   assoc.obj
 0001:0002a69c       AssocStateMachineInit      1002b69c f   assoc.obj
 0001:0002a958       MlmeAuthReqAction          1002b958 f   auth.obj
 0001:0002acb0       PeerAuthRspAtSeq2Action    1002bcb0 f   auth.obj
 0001:0002b0a8       PeerAuthRspAtSeq4Action    1002c0a8 f   auth.obj
 0001:0002b1d4       MlmeDeauthReqAction        1002c1d4 f   auth.obj
 0001:0002b360       AuthTimeoutAction          1002c360 f   auth.obj
 0001:0002b3a0       InvalidStateWhenAuth       1002c3a0 f   auth.obj
 0001:0002b3e8       Cls2errAction              1002c3e8 f   auth.obj
 0001:0002b518       AuthTimeout                1002c518 f   auth.obj
 0001:0002b594       AuthStateMachineInit       1002c594 f   auth.obj
 0001:0002b6ac       PeerDeauthAction           1002c6ac f   auth_rsp.obj
 0001:0002b8fc       AuthRspStateMachineInit    1002c8fc f   auth_rsp.obj
 0001:0002b988       MlmeCntlInit               1002c988 f   connect.obj
 0001:0002b998       SSIDIsValid                1002c998 f   connect.obj
 0001:0002b9e8       CntlWscIterate             1002c9e8 f   connect.obj
 0001:0002bab4       CntlChannelWidth           1002cab4 f   connect.obj
 0001:0002bd90       LinkDown                   1002cd90 f   connect.obj
 0001:0002c6d0       MlmeCntlConfirm            1002d6d0 f   connect.obj
 0001:0002c704       AssocParmFill              1002d704 f   connect.obj
 0001:0002c784       ScanParmFill               1002d784 f   connect.obj
 0001:0002c7bc       DlsParmFill                1002d7bc f   connect.obj
 0001:0002c7c8       TdlsParmFill               1002d7c8 f   connect.obj
 0001:0002c7d4       DisassocParmFill           1002d7d4 f   connect.obj
 0001:0002c834       DeauthParmFill             1002d834 f   connect.obj
 0001:0002c894       StartParmFill              1002d894 f   connect.obj
 0001:0002c8e0       AuthParmFill               1002d8e0 f   connect.obj
 0001:0002c948       ComposePsPoll              1002d948 f   connect.obj
 0001:0002cb5c       ComposeNullFrame           1002db5c f   connect.obj
 0001:0002cdac       MakeIbssBeacon             1002ddac f   connect.obj
 0001:0002d58c       CntlOidScanProc            1002e58c f   connect.obj
 0001:0002d7f8       CntlOidRTBssidProc         1002e7f8 f   connect.obj
 0001:0002dccc       CntlOidDLSSetupProc        1002eccc f   connect.obj
 0001:0002e0b0       CntlWaitAuthProc           1002f0b0 f   connect.obj
 0001:0002e238       CntlOidTDLSRequestProc     1002f238 f   connect.obj
 0001:0002e440       LinkUp                     1002f440 f   connect.obj
 0001:0002ff94       IterateOnBssTab            10030f94 f   connect.obj
 0001:00030330       IterateOnBssTab2           10031330 f   connect.obj
 0001:00030438       CntlOidSsidProc            10031438 f   connect.obj
 0001:00030b28       CntlMlmeRoamingProc        10031b28 f   connect.obj
 0001:00030c34       CntlWaitDisassocProc       10031c34 f   connect.obj
 0001:00030d28       CntlWaitJoinProc           10031d28 f   connect.obj
 0001:00030f9c       CntlWaitStartProc          10031f9c f   connect.obj
 0001:00031060       CntlWaitAuthProc2          10032060 f   connect.obj
 0001:0003124c       CntlWaitAssocProc          1003224c f   connect.obj
 0001:0003133c       CntlWaitReassocProc        1003233c f   connect.obj
 0001:0003144c       CntlIdleProc               1003244c f   connect.obj
 0001:00031658       MlmeCntlMachinePerformAction 10032658 f   connect.obj
 0001:00031a00       MlmeDlsReqAction           10032a00 f   dls.obj
 0001:00031cc8       PeerDlsReqAction           10032cc8 f   dls.obj
 0001:00032410       RTMPCheckDLSTimeOut        10033410 f   dls.obj
 0001:000325a8       RTMPCheckDLSFrame          100335a8 f   dls.obj
 0001:000326b4       RTMPSendDLSTearDownFrame   100336b4 f   dls.obj
 0001:000327d0       RTMPSendSTAKeyRequest      100337d0 f   dls.obj
 0001:00032c50       RTMPSendSTAKeyHandShake    10033c50 f   dls.obj
 0001:000330c8       DlsTimeout                 100340c8 f   dls.obj
 0001:0003314c       PeerDlsRspAction           1003414c f   dls.obj
 0001:000335c0       MlmeDlsTearDownAction      100345c0 f   dls.obj
 0001:0003381c       PeerDlsTearDownAction      1003481c f   dls.obj
 0001:000339cc       RTMPRcvFrameDLSCheck       100349cc f   dls.obj
 0001:00033fb0       DlsTearDown                10034fb0 f   dls.obj
 0001:000340c4       DlsStateMachineInit        100350c4 f   dls.obj
 0001:000341e4       RogueApTableInit           100351e4 f   leap.obj
 0001:00034204       RogueApTableSearch         10035204 f   leap.obj
 0001:00034264       RogueApEntrySet            10035264 f   leap.obj
 0001:000342cc       RogueApTableSetEntry       100352cc f   leap.obj
 0001:0003435c       RogueApTableDeleteEntry    1003535c f   leap.obj
 0001:00034410       LeapSendRogueAPReport      10035410 f   leap.obj
 0001:00034444       CCXAAPReasonCodeReport     10035444 f   leap.obj
 0001:0003469c       CCXAdjacentAPReport        1003569c f   leap.obj
 0001:00034ae8       MD5Transform               10035ae8 f   md5.obj
 0001:00035510       SHAInit                    10036510 f   md5.obj
 0001:000357ac       SHAUpdate                  100367ac f   md5.obj
 0001:0003587c       SHAFinal                   1003687c f   md5.obj
 0001:00035970       SHA256_Init                10036970 f   md5.obj
 0001:000359b0       SHA256_Hash                100369b0 f   md5.obj
 0001:00035bf0       SHA256_Append              10036bf0 f   md5.obj
 0001:00035c90       SHA256_End                 10036c90 f   md5.obj
 0001:00035dc0       SHA256                     10036dc0 f   md5.obj
 0001:00035e60       aes_set_key                10036e60 f   md5.obj
 0001:000363d8       aes_encrypt                100373d8 f   md5.obj
 0001:00037bb0       aes_decrypt                10038bb0 f   md5.obj
 0001:00039370       leftshift_onebit           1003a370 f   md5.obj
 0001:000393b8       do_padding                 1003a3b8 f   md5.obj
 0001:00039404       generate_subkey            1003a404 f   md5.obj
 0001:000395b4       AES_128_CMAC               1003a5b4 f   md5.obj
 0001:000397c0       MD5Update                  1003a7c0 f   md5.obj
 0001:00039888       MD5Final                   1003a888 f   md5.obj
 0001:00039930       hmac_md5                   1003a930 f   md5.obj
 0001:00039af8       MlmePeriodicExec           1003aaf8 f   mlme.obj
 0001:00039f20       LinkDownExec               1003af20 f   mlme.obj
 0001:00039f6c       LinkUpExec                 1003af6c f   mlme.obj
 0001:00039fb8       MlmeValidateSSID           1003afb8 f   mlme.obj
 0001:00039ffc       MlmeUpdateLimitTxRateTable 1003affc f   mlme.obj
 0001:0003a120       MlmeSetPsm                 1003b120 f   mlme.obj
 0001:0003a188       MlmeSetTxPreamble          1003b188 f   mlme.obj
 0001:0003a1f8       MlmeUpdateTxRates          1003b1f8 f   mlme.obj
 0001:0003ab54       MlmeUpdateHtTxRates        1003bb54 f   mlme.obj
 0001:0003af5c       AsicUpdateAutoFallBackTable 1003bf5c f   mlme.obj
 0001:0003b2bc       AsicUpdateProtect          1003c2bc f   mlme.obj
 0001:0003b58c       BssTableInit               1003c58c f   mlme.obj
 0001:0003b5b8       BATableInit                1003c5b8 f   mlme.obj
 0001:0003b5f4       BssTableSearch             1003c5f4 f   mlme.obj
 0001:0003b898       BssSsidTableSearch         1003c898 f   mlme.obj
 0001:0003b968       BssTableSearchWithSSID     1003c968 f   mlme.obj
 0001:0003ba6c       BssTableDeleteEntry        1003ca6c f   mlme.obj
 0001:0003bb54       BssTableDeleteEntryByBssid 1003cb54 f   mlme.obj
 0001:0003bbcc       BssTableDeleteEntryByChannel 1003cbcc f   mlme.obj
 0001:0003bcd8       BATableDeleteORIEntry      1003ccd8 f   mlme.obj
 0001:0003bdb8       BATableDeleteRECEntry      1003cdb8 f   mlme.obj
 0001:0003c014       BATableInsertEntry         1003d014 f   mlme.obj
 0001:0003c368       TriEventInit               1003d368 f   mlme.obj
 0001:0003c3b0       TriEventTableSetEntry      1003d3b0 f   mlme.obj
 0001:0003c4d0       BssTableSortByRssi         1003d4d0 f   mlme.obj
 0001:0003c66c       BssCipherParse             1003d66c f   mlme.obj
 0001:0003ce28       MgtMacHeaderInit           1003de28 f   mlme.obj
 0001:0003cf74       MakeOutgoingFrame          1003df74 f   mlme.obj
 0001:0003cfd4       MlmeQueueInit              1003dfd4 f   mlme.obj
 0001:0003d028       MlmeDequeue                1003e028 f   mlme.obj
 0001:0003d09c       MlmeRestartStateMachine    1003e09c f   mlme.obj
 0001:0003d2c0       MlmeQueueEmpty             1003e2c0 f   mlme.obj
 0001:0003d2f4       MlmeQueueFull              1003e2f4 f   mlme.obj
 0001:0003d33c       MlmeQueueClean             1003e33c f   mlme.obj
 0001:0003d3c0       MlmeQueueDestroy           1003e3c0 f   mlme.obj
 0001:0003d3f8       MsgTypeSubst               1003e3f8 f   mlme.obj
 0001:0003d7ac       StateMachineInit           1003e7ac f   mlme.obj
 0001:0003d818       StateMachineSetAction      1003e818 f   mlme.obj
 0001:0003d848       StateMachinePerformAction  1003e848 f   mlme.obj
 0001:0003d884       Drop                       1003e884 f   mlme.obj
 0001:0003d888       LfsrInit                   1003e888 f   mlme.obj
 0001:0003d8a0       RandomByte                 1003e8a0 f   mlme.obj
 0001:0003d8f4       AsicLockChannel            1003e8f4 f   mlme.obj
 0001:0003d8f8       AsicSetBssid               1003e8f8 f   mlme.obj
 0001:0003d9ac       AsicSetMcastWC             1003e9ac f   mlme.obj
 0001:0003d9e8       AsicDelWcidTab             1003e9e8 f   mlme.obj
 0001:0003da2c       AsicDisableSync            1003ea2c f   mlme.obj
 0001:0003da78       AsicEnableRDG              1003ea78 f   mlme.obj
 0001:0003dae4       AsicDisableRDG             1003eae4 f   mlme.obj
 0001:0003db60       AsicEnablePiggyB           1003eb60 f   mlme.obj
 0001:0003dba0       AsicDisablePiggyB          1003eba0 f   mlme.obj
 0001:0003dbe0       AsicEnableBssSync          1003ebe0 f   mlme.obj
 0001:0003dc70       AsicEnableIbssSync         1003ec70 f   mlme.obj
 0001:0003dde4       AsicSetEdcaParm            1003ede4 f   mlme.obj
 0001:0003e1c8       AsicSetSlotTime            1003f1c8 f   mlme.obj
 0001:0003e2a8       AsicBbpTuning              1003f2a8 f   mlme.obj
 0001:0003e680       AsicUpdateWCIDAttribute    1003f680 f   mlme.obj
 0001:0003e6d4       AsicUpdateWCIDIVEIV        1003f6d4 f   mlme.obj
 0001:0003e718       AsicUpdateRxWCIDTable      1003f718 f   mlme.obj
 0001:0003e788       AsicAddKeyEntry            1003f788 f   mlme.obj
 0001:0003e9d4       AsicAddSharedKeyEntry      1003f9d4 f   mlme.obj
 0001:0003eba4       AsicRemoveKeyEntry         1003fba4 f   mlme.obj
 0001:0003ebc8       AsicRemoveSharedKeyEntry   1003fbc8 f   mlme.obj
 0001:0003ec90       AsicRemovePairwiseKeyEntry 1003fc90 f   mlme.obj
 0001:0003ec94       AsicSendCommanToMcu        1003fc94 f   mlme.obj
 0001:0003ed48       RTMPCheckRates             1003fd48 f   mlme.obj
 0001:0003ee5c       RTMPCheckChannel           1003fe5c f   mlme.obj
 0001:0003ef1c       RTMPCheckHt                1003ff1c f   mlme.obj
 0001:0003f498       AsicSetRxAnt               10040498 f   mlme.obj
 0001:0003f56c       AsicEvaluateRxAnt          1004056c f   mlme.obj
 0001:0003f708       AsicRxAntEvalTimeout       10040708 f   mlme.obj
 0001:0003f72c       AsicRxAntEvalAction        1004072c f   mlme.obj
 0001:0003f8e8       RadarDetectionStart        100408e8 f   mlme.obj
 0001:0003f8ec       RadarDetectionStop         100408ec f   mlme.obj
 0001:0003f8fc       RadarChannelCheck          100408fc f   mlme.obj
 0001:0003f9e8       MlmeFreeMemory             100409e8 f   mlme.obj
 0001:0003fc20       MlmeAllocateMemory         10040c20 f   mlme.obj
 0001:0003fd18       MlmeInitMemoryHandler      10040d18 f   mlme.obj
 0001:0003fe9c       MlmeFreeMemoryHandler      10040e9c f   mlme.obj
 0001:0003ff3c       RTMPUpdateMlmeRate         10040f3c f   mlme.obj
 0001:00040140       RTMPMaxRssi                10041140 f   mlme.obj
 0001:000401a0       RTMPSetAGCInitValue        100411a0 f   mlme.obj
 0001:00040310       CarrierDetectTimeout       10041310 f   mlme.obj
 0001:0004033c       AsicSendNullFrame          1004133c f   mlme.obj
 0001:00040748       RTUSBFilterCalibration     10041748 f   mlme.obj
 0001:00040a84       SSIDLUpdateBssEntry        10041a84 f   mlme.obj
 0001:00040ed8       AsicCheckCommandOk         10041ed8 f   mlme.obj
 0001:00040fe8       InitDesiredTSSITable       10041fe8 f   mlme.obj
 0001:0004154c       GetDesiredTSSI             1004254c f   mlme.obj
 0001:0004160c       MlmeInit                   1004260c f   mlme.obj
 0001:000419d4       MlmeHalt                   100429d4 f   mlme.obj
 0001:00041c2c       MlmeCalculateChannelQuality 10042c2c f   mlme.obj
 0001:00041df4       MlmeSetTxRate              10042df4 f   mlme.obj
 0001:0004269c       MlmeSelectTxRateTable      1004369c f   mlme.obj
 0001:00042fc8       MlmeDynamicTxRateSwitching 10043fc8 f   mlme.obj
 0001:00044358       StaQuickResponeForRateUpExec 10045358 f   mlme.obj
 0001:00044874       MlmeCheckPsmChange         10045874 f   mlme.obj
 0001:00044930       MlmeRadioOff               10045930 f   mlme.obj
 0001:00044ccc       BssEntrySet                10045ccc f   mlme.obj
 0001:00045148       BssTableSetEntry           10046148 f   mlme.obj
 0001:000455fc       BssTableSsidSort           100465fc f   mlme.obj
 0001:00045ae4       MacAddrRandomBssid         10046ae4 f   mlme.obj
 0001:00045b24       MlmeEnqueue                10046b24 f   mlme.obj
 0001:00045c00       MlmeEnqueueForRecv         10046c00 f   mlme.obj
 0001:00045d64       AsicSwitchChannel          10046d64 f   mlme.obj
 0001:00046c54       AsicAdjustTxPower          10047c54 f   mlme.obj
 0001:000476f8       AsicSleepThenAutoWakeup    100486f8 f   mlme.obj
 0001:00047778       AsicForceWakeup            10048778 f   mlme.obj
 0001:000477cc       AsicSetCarrierDetectAction 100487cc f   mlme.obj
 0001:0004782c       CarrierDetectTimeoutAction 1004882c f   mlme.obj
 0001:00047a3c       AsicSendBA                 10048a3c f   mlme.obj
 0001:00047dcc       MlmeAutoScan               10048dcc f   mlme.obj
 0001:00047e30       MlmeAutoReconnectLastSSID  10048e30 f   mlme.obj
 0001:00047f20       MlmeCheckForFastRoaming    10048f20 f   mlme.obj
 0001:0004850c       MlmeRadioOn                1004950c f   mlme.obj
 0001:000486bc       BATableTearRECEntry        100496bc f   mlme.obj
 0001:000488f0       BATableTearORIEntry        100498f0 f   mlme.obj
 0001:00048b98       MlmePostRestartStateMachine 10049b98 f   mlme.obj
 0001:00048c34       MlmeHandler                10049c34 f   mlme.obj
 0001:00048e84       STAMlmePeriodicExec        10049e84 f   mlme.obj
 0001:0004a828       MlmeThread                 1004b828 f   mlme.obj
 0001:0004a89c       next_key@8                 1004b89c f i rtmp_ckipmic.obj
 0001:0004a928       byte_sub_shift_row@8       1004b928 f i rtmp_ckipmic.obj
 0001:0004a9fc       CKIP_key_permute           1004b9fc f   rtmp_ckipmic.obj
 0001:0004ab90       mix_column_DWORD32         1004bb90 f   rtmp_ckipmic.obj
 0001:0004abe4       RTMPCkipDecrypt            1004bbe4 f   rtmp_ckipmic.obj
 0001:0004ad4c       RTMPAesEncrypt             1004bd4c f i rtmp_ckipmic.obj
 0001:0004aeb4       RTMPMicGetCoefficient      1004beb4 f i rtmp_ckipmic.obj
 0001:0004af60       RTMPMicUpdate              1004bf60 f i rtmp_ckipmic.obj
 0001:0004b020       RTMPMicFinal               1004c020 f i rtmp_ckipmic.obj
 0001:0004b140       RTMPCkipInsertCMIC         1004c140 f   rtmp_ckipmic.obj
 0001:0004b3c4       RTMPCkipCalCMIC            1004c3c4 f   rtmp_ckipmic.obj
 0001:0004b5c8       BtCheckWifiThroughputOverLimit 1004c5c8 f   rtmp_cobt.obj
 0001:0004b69c       BtCheckBusy                1004c69c f   rtmp_cobt.obj
 0001:0004b87c       BtCoexistDetectExecAtCmdThread 1004c87c f   rtmp_cobt.obj
 0001:0004bdb8       BtCoexistDetectExecAtTimer 1004cdb8 f   rtmp_cobt.obj
 0001:0004be84       InitBTCoexistence          1004ce84 f   rtmp_cobt.obj
 0001:0004c088       RTMPWPARemoveKeyProc       1004d088 f   rtmp_info.obj
 0001:0004c184       RTMPWPARemoveAllKeys       1004d184 f   rtmp_info.obj
 0001:0004c1d8       RTMPIndicateWPA2Status     1004d1d8 f   rtmp_info.obj
 0001:0004c30c       RTMPOPModeSwitching        1004d30c f   rtmp_info.obj
 0001:0004c43c       RTMPAddBSSIDCipher         1004d43c f   rtmp_info.obj
 0001:0004c900       RTMPSetHT                  1004d900 f   rtmp_info.obj
 0001:0004d398       RTMPUpdateHTIE             1004e398 f   rtmp_info.obj
 0001:0004d5ac       LEDConnectionStart         1004e5ac f   rtmp_info.obj
 0001:0004d624       LEDConnectionCompletion    1004e624 f   rtmp_info.obj
 0001:0004d6b0       RTMPMantainAdhocList       1004e6b0 f   rtmp_info.obj
 0001:0004d794       STASetInformation          1004e794 f   rtmp_info.obj
 0001:000513dc       RTMPWPAAddKeyProc          100523dc f   rtmp_info.obj
 0001:00051e28       RTMPSetPhyMode             10052e28 f   rtmp_info.obj
 0001:00052328       RTMPSetInformation         10053328 f   rtmp_info.obj
 0001:000531f4       STAQueryInformation        100541f4 f   rtmp_info.obj
 0001:0005516c       RTMPQueryInformation       1005616c f   rtmp_info.obj
 0001:000570b8       BitReverse                 100580b8 f   rtmp_init.obj
 0001:000570ec       RTMPAllocAdapterBlock      100580ec f   rtmp_init.obj
 0001:00057154       NICInitTransmit            10058154 f   rtmp_init.obj
 0001:00057584       CreateThreads              10058584 f   rtmp_init.obj
 0001:0005766c       NICInitRecv                1005866c f   rtmp_init.obj
 0001:000577b0       RTUSBKickbulkoutDPC        100587b0 f   rtmp_init.obj
 0001:00057834       FreeNICRecv                10058834 f   rtmp_init.obj
 0001:000578f0       FreeNICTransmit            100588f0 f   rtmp_init.obj
 0001:00057afc       DisallocateAllSpinLock     10058afc f   rtmp_init.obj
 0001:00057cdc       RTMPInitAdapterBlock       10058cdc f   rtmp_init.obj
 0001:0005803c       ReleaseAdapter             1005903c f   rtmp_init.obj
 0001:0005807c       RTMPReadTxPwrPerRate       1005907c f   rtmp_init.obj
 0001:000585bc       RTMPReadChannelPwr         100595bc f   rtmp_init.obj
 0001:00058b14       RTUSBWriteHWMACAddress     10059b14 f   rtmp_init.obj
 0001:00058bdc       NICReadEEPROMParameters    10059bdc f   rtmp_init.obj
 0001:00059440       RT30xxInitAsic             1005a440 f   rtmp_init.obj
 0001:00059d90       PostBBPInitialization      1005ad90 f   rtmp_init.obj
 0001:00059e84       PostRFInitialization       1005ae84 f   rtmp_init.obj
 0001:00059f44       NICWaitMACReady            1005af44 f   rtmp_init.obj
 0001:00059f98       NICInitializeAsic          1005af98 f   rtmp_init.obj
 0001:0005a628       NICUpdateRawCounters       1005b628 f   rtmp_init.obj
 0001:0005a7cc       RTMPEqualMemory            1005b7cc f   rtmp_init.obj
 0001:0005a818       RTMPCompareMemory          1005b818 f   rtmp_init.obj
 0001:0005a874       RTMPZeroMemory             1005b874 f   rtmp_init.obj
 0001:0005a894       RTMPMoveMemory             1005b894 f   rtmp_init.obj
 0001:0005a8b4       UserCfgInit                1005b8b4 f   rtmp_init.obj
 0001:0005af8c       EnableTwoPhasesScanOperation 1005bf8c f   rtmp_init.obj
 0001:0005afc8       BtoH                       1005bfc8 f   rtmp_init.obj
 0001:0005b018       AtoH                       1005c018 f   rtmp_init.obj
 0001:0005b060       RTMPInitTimer              1005c060 f   rtmp_init.obj
 0001:0005b094       RTMPSetTimer               1005c094 f   rtmp_init.obj
 0001:0005b0f0       RTMPCancelTimer            1005c0f0 f   rtmp_init.obj
 0001:0005b12c       RTMPSetLED                 1005c12c f   rtmp_init.obj
 0001:0005b5d4       RTMPSetSignalLED           1005c5d4 f   rtmp_init.obj
 0001:0005b674       RTMPEnableRxTx             1005c674 f   rtmp_init.obj
 0001:0005b7bc       RTMPReadSafelyRemoveFlag   1005c7bc f   rtmp_init.obj
 0001:0005b884       RTMPPrepareCTSFrame        1005c884 f   rtmp_init.obj
 0001:0005ba2c       RTMPSetMessageEvent        1005ca2c f   rtmp_init.obj
 0001:0005bbdc       AsicRadioOff               1005cbdc f   rtmp_init.obj
 0001:0005be44       AsicRFOn                   1005ce44 f   rtmp_init.obj
 0001:0005c078       AsicRadioOn                1005d078 f   rtmp_init.obj
 0001:0005c17c       IsRalinkEncStr             1005d17c f   rtmp_init.obj
 0001:0005c240       DecryptWepRegistry         1005d240 f   rtmp_init.obj
 0001:0005c328       NICReadRegParameters       1005d328 f   rtmp_init.obj
 0001:0005cb24       NICInitAsicFromEEPROM      1005db24 f   rtmp_init.obj
 0001:0005d2b8       NICResetFromError          1005e2b8 f   rtmp_init.obj
 0001:0005d2ec       NICLoadFirmware            1005e2ec f   rtmp_init.obj
 0001:0005d6b4       RTMPInitialize             1005e6b4 f   rtmp_main.obj
 0001:0005dba0       RTMPCheckForHang           1005eba0 f   rtmp_main.obj
 0001:0005dc20       RTMPHalt                   1005ec20 f   rtmp_main.obj
 0001:0005dfd0       RTMPReset                  1005efd0 f   rtmp_main.obj
 0001:0005dff0       RTMPTransferData           1005eff0 f   rtmp_main.obj
 0001:0005e0e8       RTMPPnPEventNotify         1005f0e8 f   rtmp_main.obj
 0001:0005e194       RTMPShutdown               1005f194 f   rtmp_main.obj
 0001:0005e208       JunkThread                 1005f208 f   rtmp_main.obj
 0001:0005e36c       DriverEntry                1005f36c f   rtmp_main.obj
 0001:0005e4a8       byte_sub                   1005f4a8 f i rtmp_tkip.obj
 0001:0005e574       shift_row                  1005f574 f i rtmp_tkip.obj
 0001:0005e5f8       mix_column                 1005f5f8 f i rtmp_tkip.obj
 0001:0005e6c4       RTMPTkipSetMICKey          1005f6c4 f   rtmp_tkip.obj
 0001:0005e738       RTMPTkipAppendByte         1005f738 f   rtmp_tkip.obj
 0001:0005e7e8       RTMPTkipAppend             1005f7e8 f   rtmp_tkip.obj
 0001:0005e818       RTMPTkipGetMIC             1005f818 f   rtmp_tkip.obj
 0001:0005e8a4       RTMPInitTkipEngine         1005f8a4 f   rtmp_tkip.obj
 0001:0005e928       RTMPInitMICEngine          1005f928 f   rtmp_tkip.obj
 0001:0005e9b8       RTMPTkipCompareMICValue    1005f9b8 f   rtmp_tkip.obj
 0001:0005eacc       RTMPCalculateMICValue      1005facc f   rtmp_tkip.obj
 0001:0005ebd4       RTMPTkipMixKey             1005fbd4 f   rtmp_tkip.obj
 0001:0005f190       construct_mic_header1      10060190 f   rtmp_tkip.obj
 0001:0005f234       construct_mic_header2      10060234 f   rtmp_tkip.obj
 0001:0005f324       construct_mic_iv           10060324 f   rtmp_tkip.obj
 0001:0005f3d4       aes128k128d                100603d4 f   rtmp_tkip.obj
 0001:0005f560       construct_ctr_preload      10060560 f   rtmp_tkip.obj
 0001:0005f61c       GetMacHdrLength            1006061c f   rtmp_tkip.obj
 0001:0005f6dc       RTMPSoftEncryptTKIP        100606dc f   rtmp_tkip.obj
 0001:0005fa94       RTMPSoftDecryptTKIP        10060a94 f   rtmp_tkip.obj
 0001:0005fde0       RTMPSoftEncryptAES         10060de0 f   rtmp_tkip.obj
 0001:00060364       RTMPSoftDecryptAES         10061364 f   rtmp_tkip.obj
 0001:00060848       ccmp128_init               10061848 f   rtmp_tkip.obj
 0001:00060ef0       ccmp128_encrypt            10061ef0 f   rtmp_tkip.obj
 0001:00061360       ccmp128_decrypt            10062360 f   rtmp_tkip.obj
 0001:000617d0       ccmp128_finalize           100627d0 f   rtmp_tkip.obj
 0001:00061914       RTMPSoftEncryptMgmtAES     10062914 f   rtmp_tkip.obj
 0001:00061c64       RTMPSoftDecryptMgmtAES     10062c64 f   rtmp_tkip.obj
 0001:00061f08       ARCFOUR_INIT               10062f08 f   rtmp_wep.obj
 0001:00061f90       ARCFOUR_BYTE               10062f90 f   rtmp_wep.obj
 0001:00061fe4       ARCFOUR_DECRYPT            10062fe4 f   rtmp_wep.obj
 0001:00062058       ARCFOUR_ENCRYPT            10063058 f   rtmp_wep.obj
 0001:000620cc       WPAARCFOUR_ENCRYPT         100630cc f   rtmp_wep.obj
 0001:00062190       RTMP_CALC_FCS32            10063190 f   rtmp_wep.obj
 0001:000621c8       RTMPSetICV                 100631c8 f   rtmp_wep.obj
 0001:00062204       RTMPInitWepEngine          10063204 f   rtmp_wep.obj
 0001:000622dc       RTMPEncryptData            100632dc f   rtmp_wep.obj
 0001:0006232c       RTMPDecryptData            1006332c f   rtmp_wep.obj
 0001:0006248c       RTUSBInitHTTxDesc          1006348c f   rtusb_bulk.obj
 0001:00062490       RTUSBComposeUnit           10063490 f   rtusb_bulk.obj
 0001:00062c9c       RTUSBBulkOutDataPacketComplete 10063c9c f   rtusb_bulk.obj
 0001:00062e24       RTUSBBulkOutNullFrameComplete 10063e24 f   rtusb_bulk.obj
 0001:00062f4c       RTUSBBulkOutMLMEPacketComplete 10063f4c f   rtusb_bulk.obj
 0001:0006315c       RTUSBBulkOutPsPollComplete 1006415c f   rtusb_bulk.obj
 0001:00063284       RTUSBBulkReceive           10064284 f   rtusb_bulk.obj
 0001:00063450       RTUSBBulkRxComplete        10064450 f   rtusb_bulk.obj
 0001:00063624       RTUSBCleanUpDataBulkOutQueue 10064624 f   rtusb_bulk.obj
 0001:000636a8       RTUSBCleanUpMLMEBulkOutQueue 100646a8 f   rtusb_bulk.obj
 0001:00063754       RTUSBCancelPendingBulkInIRP 10064754 f   rtusb_bulk.obj
 0001:00063788       RTUSBCancelPendingBulkOutIRP 10064788 f   rtusb_bulk.obj
 0001:00063900       RTUSBBulkOutDataPacket     10064900 f   rtusb_bulk.obj
 0001:00063d04       RTUSBBulkOutNullFrame      10064d04 f   rtusb_bulk.obj
 0001:00063e08       RTUSBBulkOutMLMEPacket     10064e08 f   rtusb_bulk.obj
 0001:00063f24       RTUSBBulkOutPsPoll         10064f24 f   rtusb_bulk.obj
 0001:00064014       RTUSBKickBulkOut           10065014 f   rtusb_bulk.obj
 0001:000642c8       RTUSBCancelPendingIRPs     100652c8 f   rtusb_bulk.obj
 0001:000642e4       Sniff2BytesFromNdisBuffer  100652e4 f   rtusb_data.obj
 0001:00064368       RTUSBFreeDescriptorRequest 10065368 f   rtusb_data.obj
 0001:00064484       RTUSBSuspendMsduTransmission 10065484 f   rtusb_data.obj
 0001:00064534       RTUSBCalcDuration          10065534 f   rtusb_data.obj
 0001:000645f4       RTMPWriteTxWI              100655f4 f   rtusb_data.obj
 0001:00064900       RTMPWriteTxInfo            10065900 f   rtusb_data.obj
 0001:00064958       TxFrameIsAggregatible      10065958 f   rtusb_data.obj
 0001:000649d0       RTMPFreeNdisPacket         100659d0 f   rtusb_data.obj
 0001:00064a24       RTMPDecideSegmentEnd       10065a24 f   rtusb_data.obj
 0001:00064a88       RTUSBCleanUpMLMEWaitQueue  10065a88 f   rtusb_data.obj
 0001:00064b64       RTMPApplyPacketFilter      10065b64 f   rtusb_data.obj
 0001:00064c88       RTUSBMlmeHardTransmit      10065c88 f   rtusb_data.obj
 0001:00065220       RTMPCalcDuration           10066220 f   rtusb_data.obj
 0001:000652ec       RTMPCheckDHCPFrame         100662ec f   rtusb_data.obj
 0001:000653f0       RTMPCheckTxSIPPacket       100663f0 f   rtusb_data.obj
 0001:000655fc       RTMPCheckRxSIPPacket       100665fc f   rtusb_data.obj
 0001:00065754       RTMPSearchTupleCache       10066754 f   rtusb_data.obj
 0001:000657e0       RTMPUpdateTupleCache       100667e0 f   rtusb_data.obj
 0001:00065924       MulticastRate_NRateToOFDMRate 10066924 f   rtusb_data.obj
 0001:00065a5c       RTMPSendBAR                10066a5c f   rtusb_data.obj
 0001:00065f70       MCSToPhyRateIn500kps       10066f70 f   rtusb_data.obj
 0001:000662b4       RTMPSendPacket             100672b4 f   rtusb_data.obj
 0001:00066784       RTUSBRejectPendingPackets  10067784 f   rtusb_data.obj
 0001:00066938       RTUSBHardTransmit          10067938 f   rtusb_data.obj
 0001:000696d0       RTUSBDequeueMLMEPacket     1006a6d0 f   rtusb_data.obj
 0001:00069844       MiniportMMRequest          1006a844 f   rtusb_data.obj
 0001:00069a48       RTMPReportMicError         1006aa48 f   rtusb_data.obj
 0001:00069b6c       RTMPSendNullFrame          1006ab6c f   rtusb_data.obj
 0001:0006a064       RTMPSendNullFrameForDirect 1006b064 f   rtusb_data.obj
 0001:0006a4e0       RTMPDeQueuePacket          1006b4e0 f   rtusb_data.obj
 0001:0006a798       RTUSBResumeMsduTransmission 1006b798 f   rtusb_data.obj
 0001:0006a94c       RTMPCheckRxWI              1006b94c f   rtusb_data.obj
 0001:0006ae18       RTMPSendTxWaitQueue        1006be18 f   rtusb_data.obj
 0001:0006b0c8       RTMPSendPackets            1006c0c8 f   rtusb_data.obj
 0001:0006b30c       RTUSBRxPacket              1006c30c f   rtusb_data.obj
 0001:0006d954       InitEFuseConfig            1006e954 f   rtusb_io.obj
 0001:0006d9dc       RTUSBInitializeCmdQ        1006e9dc f   rtusb_io.obj
 0001:0006d9f0       RTUSBEnqueueCmdFromNdis    1006e9f0 f   rtusb_io.obj
 0001:0006dc24       RTUSBEnqueueInternalCmd    1006ec24 f   rtusb_io.obj
 0001:0006dd94       RTUSBDequeueCmd            1006ed94 f   rtusb_io.obj
 0001:0006ddc8       RTUSB_VendorRequest        1006edc8 f   rtusb_io.obj
 0001:0006dff4       RTUSB_InterfaceStop        1006eff4 f   rtusb_io.obj
 0001:0006dff8       RTUSB_ResetPipe            1006eff8 f   rtusb_io.obj
 0001:0006e0f4       RTUSB_AbortPipe            1006f0f4 f   rtusb_io.obj
 0001:0006e160       RTUSB_GetPortStatus        1006f160 f   rtusb_io.obj
 0001:0006e170       RTUSB_EndpointUsage        1006f170 f   rtusb_io.obj
 0001:0006e228       RTUSB_ReBulkOut            1006f228 f   rtusb_io.obj
 0001:0006e374       RTUSBFirmwareRun           1006f374 f   rtusb_io.obj
 0001:0006e3b0       RTUSBFirmwareOpmode        1006f3b0 f   rtusb_io.obj
 0001:0006e3f4       RTUSBVenderReset           1006f3f4 f   rtusb_io.obj
 0001:0006e430       RTUSBSingleWrite           1006f430 f   rtusb_io.obj
 0001:0006e470       RTUSBMultiRead             1006f470 f   rtusb_io.obj
 0001:0006e4b4       RTUSBMultiWrite2           1006f4b4 f   rtusb_io.obj
 0001:0006e4f8       RTUSBMultiWrite            1006f4f8 f   rtusb_io.obj
 0001:0006e574       RTUSBReadMACRegister       1006f574 f   rtusb_io.obj
 0001:0006e5b8       RTUSBWriteMACRegister      1006f5b8 f   rtusb_io.obj
 0001:0006e624       RTUSBReadBBPRegister       1006f624 f   rtusb_io.obj
 0001:0006e718       RTUSBWriteBBPRegister      1006f718 f   rtusb_io.obj
 0001:0006e7cc       RTUSBWriteRFRegister       1006f7cc f   rtusb_io.obj
 0001:0006e85c       RT30xxWriteRFRegister      1006f85c f   rtusb_io.obj
 0001:0006e90c       RT3572WriteBBPR66          1006f90c f   rtusb_io.obj
 0001:0006e9c0       RT30xxReadRFRegister       1006f9c0 f   rtusb_io.obj
 0001:0006ea88       eFusePhysicalReadRegisters 1006fa88 f   rtusb_io.obj
 0001:0006eb90       eFuseReadRegisters         1006fb90 f   rtusb_io.obj
 0001:0006ecbc       eFuseRead                  1006fcbc f   rtusb_io.obj
 0001:0006ed18       eFuseReadPhysical          1006fd18 f   rtusb_io.obj
 0001:0006ed70       eFusePhysicalWriteRegisters 1006fd70 f   rtusb_io.obj
 0001:0006ef50       eFuseWritePhysical         1006ff50 f   rtusb_io.obj
 0001:0006efb0       eFuseWriteRegisters        1006ffb0 f   rtusb_io.obj
 0001:0006f5c4       eFuseWrite                 100705c4 f   rtusb_io.obj
 0001:0006f620       RTUSBWriteEEPROM           10070620 f   rtusb_io.obj
 0001:0006f664       FlashInstallationWith8KBFirmware 10070664 f   rtusb_io.obj
 0001:0006f6d4       RTUSBReadEEPROM            100706d4 f   rtusb_io.obj
 0001:0006f754       RTUSBQueryHardWareRegister 10070754 f   rtusb_io.obj
 0001:0006f914       RTUSBSetHardWareRegister   10070914 f   rtusb_io.obj
 0001:0007081c       RTUSBCmdThread             1007181c f   rtusb_io.obj
 0001:00073a40       MlmeScanReqSanity          10074a40 f   sanity.obj
 0001:00073b00       MlmeStartReqSanity         10074b00 f   sanity.obj
 0001:00073b3c       MlmeAssocReqSanity         10074b3c f   sanity.obj
 0001:00073bc4       MlmeAuthReqSanity          10074bc4 f   sanity.obj
 0001:00073c6c       PeerAssocRspSanity         10074c6c f   sanity.obj
 0001:00074178       PeerDisassocSanity         10075178 f   sanity.obj
 0001:000742b0       PeerDeauthSanity           100752b0 f   sanity.obj
 0001:000743e8       PeerAuthSanity             100753e8 f   sanity.obj
 0001:000744f8       PeerProbeReqSanity         100754f8 f   sanity.obj
 0001:000745d4       PeerBeaconAndProbeRspSanity2 100755d4 f   sanity.obj
 0001:0007468c       PeerAddBAReqActionSanity   1007568c f   sanity.obj
 0001:00074720       PeerAddBARspActionSanity   10075720 f   sanity.obj
 0001:00074750       PeerDelBAActionSanity      10075750 f   sanity.obj
 0001:00074770       GetTimBit                  10075770 f   sanity.obj
 0001:00074854       ChannelSanity              10075854 f   sanity.obj
 0001:000748ac       PeerTxTypeInUseSanity      100758ac f   sanity.obj
 0001:00074980       RTMPWPAWepKeySanity        10075980 f   sanity.obj
 0001:00074a88       RTMPRemoveKeySanity        10075a88 f   sanity.obj
 0001:00074b8c       MlmeAddBAReqSanity         10075b8c f   sanity.obj
 0001:00074bd0       MlmeDelBAReqSanity         10075bd0 f   sanity.obj
 0001:00074c00       MlmeDlsReqSanity           10075c00 f   sanity.obj
 0001:00074c24       PeerDlsReqSanity           10075c24 f   sanity.obj
 0001:00074d14       PeerDlsRspSanity           10075d14 f   sanity.obj
 0001:00074e04       PeerDlsTearDownSanity      10075e04 f   sanity.obj
 0001:00074e54       PeerAcmRspSanity           10075e54 f   sanity.obj
 0001:00074e80       MlmeTdlsReqSanity          10075e80 f   sanity.obj
 0001:00074ea4       PeerTdlsSetupReqSanity     10075ea4 f   sanity.obj
 0001:000751ac       PeerTdlsSetupRspSanity     100761ac f   sanity.obj
 0001:000754f0       PeerTdlsSetupConfSanity    100764f0 f   sanity.obj
 0001:000757f0       PeerTdlsTearDownSanity     100767f0 f   sanity.obj
 0001:00075960       PeerBeaconAndProbeRspSanity 10076960 f   sanity.obj
 0001:000767a4       NetworkTypeInUseSanity     100777a4 f   sanity.obj
 0001:00076808       STAWapiWAIPacket_HandleUnicastConf 10077808 f   Sta_wapi.obj
 0001:00076a40       STAWapiSend_MBcastKeyNegotiate_Rsp 10077a40 f   Sta_wapi.obj
 0001:00076cd0       STAWapiSend_UnicastKeyNegotiate_Rsp 10077cd0 f   Sta_wapi.obj
 0001:00076f84       STAWapi_RxSMS4Decrypt      10077f84 f   Sta_wapi.obj
 0001:00077330       STAWapiWAIPacket_HandleMBcastReq 10078330 f   Sta_wapi.obj
 0001:00077750       STAWapiWAIPacket_HandleUnicastReq 10078750 f   Sta_wapi.obj
 0001:00077948       STAWapiWAIPacketAction     10078948 f   Sta_wapi.obj
 0001:00077a8c       STAWapiStateMachineInit    10078a8c f   Sta_wapi.obj
 0001:00077aec       BeaconTimeout              10078aec f   sync.obj
 0001:00077b48       ScanTimeout                10078b48 f   sync.obj
 0001:00077ba4       InvalidStateNullFunction   10078ba4 f   sync.obj
 0001:00077bb0       MlmeJoinReqAction          10078bb0 f   sync.obj
 0001:00078194       PeerProbeReqAction         10079194 f   sync.obj
 0001:00078948       BeaconTimeoutAtJoinAction  10079948 f   sync.obj
 0001:00078a10       HasHiddenAPAtThisChannel   10079a10 f   sync.obj
 0001:00078a94       ScanNextChannel            10079a94 f   sync.obj
 0001:00079908       InvalidStateWhenJoin       1007a908 f   sync.obj
 0001:00079d20       InvalidStateWhenStart      1007ad20 f   sync.obj
 0001:00079d80       EnqueueBeaconFrame         1007ad80 f   sync.obj
 0001:00079d8c       BuildChannelList           1007ad8c f   sync.obj
 0001:0007a3c0       FirstChannel               1007b3c0 f   sync.obj
 0001:0007a3dc       NextChannel                1007b3dc f   sync.obj
 0001:0007a480       ChangeToCellPowerLimit     1007b480 f   sync.obj
 0001:0007a4e8       ConvertToRssi              1007b4e8 f   sync.obj
 0001:0007a5cc       DeleteEffectedChannelList  1007b5cc f   sync.obj
 0001:0007a630       AddToRepositList           1007b630 f   sync.obj
 0001:0007adfc       IsValidChannel             1007bdfc f   sync.obj
 0001:0007ae54       RTMPCheckBWOffset          1007be54 f   sync.obj
 0001:0007b0a8       StaAdhocUpdateMacTableEntry 1007c0a8 f   sync.obj
 0001:0007b7e4       MlmeProbeInactiveStation   1007c7e4 f   sync.obj
 0001:0007b924       MlmeScanReqAction          1007c924 f   sync.obj
 0001:0007bda0       MlmeStartReqAction         1007cda0 f   sync.obj
 0001:0007c218       PeerBeaconAtScanAction     1007d218 f   sync.obj
 0001:0007cc7c       PeerBeaconAtJoinAction     1007dc7c f   sync.obj
 0001:0007d680       ScanTimeoutAction          1007e680 f   sync.obj
 0001:0007d998       InvalidStateWhenScan       1007e998 f   sync.obj
 0001:0007dc64       BuildEffectedChannelList   1007ec64 f   sync.obj
 0001:0007dd04       PeerBeacon                 1007ed04 f   sync.obj
 0001:0007f688       SyncStateMachineInit       10080688 f   sync.obj
 0001:0007f8cc       RTUSBCE_ClosePipe          100808cc f   wince.obj
 0001:0007f908       RTUSBCE_RemoveDeviceContext 10080908 f   wince.obj
 0001:0007f9ac       RTUSBCE_DeviceNotify       100809ac f   wince.obj
 0001:0007fb00       RTUSBCE_ConfigureDevice    10080b00 f   wince.obj
 0001:0007fda0       RTUSBCE_InterfaceStart     10080da0 f   wince.obj
 0001:0007fea0       USBInstallDriver           10080ea0 f   wince.obj
 0001:0007ff70       USBUnInstallDriver         10080f70 f   wince.obj
 0001:00080018       LoadVIDFromRegistry        10081018 f   wince.obj
 0001:0008012c       ParseUsbDescriptors        1008112c f   wince.obj
 0001:000802c0       RTMPCopyUnicodeString      100812c0 f   wince.obj
 0001:0008035c       DumpSystemInfo             1008135c f   wince.obj
 0001:00080404       DllEntry                   10081404 f   wince.obj
 0001:00080490       USBDeviceAttach            10081490 f   wince.obj
 0001:00080574       WpaMsgTypeSubst            10081574 f   wpa.obj
 0001:000805d0       WpaMacHeaderInit           100815d0 f   wpa.obj
 0001:00080754       WpaHardTransmit            10081754 f   wpa.obj
 0001:00080bb8       HMAC_SHA1                  10081bb8 f   wpa.obj
 0001:00080d10       PRF                        10081d10 f   wpa.obj
 0001:00080e10       WpaCountPTK                10081e10 f   wpa.obj
 0001:00080fdc       GenRandom                  10081fdc f   wpa.obj
 0001:00081154       AES_GTK_KEY_UNWRAP         10082154 f   wpa.obj
 0001:000812a4       HMAC_SHA256                100822a4 f   wpa.obj
 0001:00081410       FT_KDF                     10082410 f   wpa.obj
 0001:00081534       WpaPairMsg1Action          10082534 f   wpa.obj
 0001:00081890       WpaPairMsg3Action          10082890 f   wpa.obj
 0001:00081d70       WpaGroupMsg1Action         10082d70 f   wpa.obj
 0001:00082284       WpaEAPOLKeyAction          10083284 f   wpa.obj
 0001:00082540       WpaPskStateMachineInit     10083540 f   wpa.obj
 0001:000825a0       WscRxMsgType               100835a0 f   wsc.obj
 0001:0008278c       WscMsgTypeSubst            1008378c f   wsc.obj
 0001:000827d4       WscConnectTimeout          100837d4 f   wsc.obj
 0001:000829a0       WscEAPRxTimeout            100839a0 f   wsc.obj
 0001:00082ad0       WscM8WaitEapFailTimeout    10083ad0 f   wsc.obj
 0001:00082b28       WscEapM2Timeout            10083b28 f   wsc.obj
 0001:00082b7c       WscSkipTurnOffLEDTimer     10083b7c f   wsc.obj
 0001:00082b94       WscScanExec                10083b94 f   wsc.obj
 0001:00082c8c       WscPBCBssTableSort         10083c8c f   wsc.obj
 0001:000832c0       WscPBCModeAPSearch         100842c0 f   wsc.obj
 0001:000837a8       WscPINModeAPSearch         100847a8 f   wsc.obj
 0001:00083c78       WscCheckWPSAP              10084c78 f   wsc.obj
 0001:00083f24       WscMacHeaderInit           10084f24 f   wsc.obj
 0001:00084080       WscStartAction             10085080 f   wsc.obj
 0001:00084284       WscInitRegistrarPair       10085284 f   wsc.obj
 0001:000846a8       MakeWSCEAPFrame            100856a8 f   wsc.obj
 0001:0008495c       WscSendEapRspId            1008595c f   wsc.obj
 0001:00084b5c       WscSendMessageM1           10085b5c f   wsc.obj
 0001:00084f84       WscSendMessageM2           10085f84 f   wsc.obj
 0001:00085594       WscSendMessageM3           10086594 f   wsc.obj
 0001:000858fc       WscSendMessageM4           100868fc f   wsc.obj
 0001:00085d90       WscSendMessageM5           10086d90 f   wsc.obj
 0001:0008609c       WscSendMessageM6           1008709c f   wsc.obj
 0001:000863bc       WscSendMessageM7           100873bc f   wsc.obj
 0001:000866c0       WscSendEapRspAck           100876c0 f   wsc.obj
 0001:000867d8       WscSendEapRspNack          100877d8 f   wsc.obj
 0001:000868f4       WscSendEapRspDone          100878f4 f   wsc.obj
 0001:000869e4       WscRecvMessageM1           100879e4 f   wsc.obj
 0001:00086dcc       WscRecvMessageM2           10087dcc f   wsc.obj
 0001:00087344       WscRecvMessageM2D          10088344 f   wsc.obj
 0001:00087474       WscRecvMessageM3           10088474 f   wsc.obj
 0001:000876d0       WscReceiveEapNack          100886d0 f   wsc.obj
 0001:00087940       WscReceiveEapDone          10088940 f   wsc.obj
 0001:00087a88       WscParseEncrSettings       10088a88 f   wsc.obj
 0001:00087e54       WscProcessCredential       10088e54 f   wsc.obj
 0001:000880d0       WscMakeProbeReqIE          100890d0 f   wsc.obj
 0001:0008830c       WscStop                    1008930c f   wsc.obj
 0001:000883d8       WscAutoGenProfile          100893d8 f   wsc.obj
 0001:000885e8       WscSupportWPSLEDMode       100895e8 f   wsc.obj
 0001:00088624       WscSupportWPSLEDMode10     10089624 f   wsc.obj
 0001:00088648       WscAPHasSecuritySetting    10089648 f   wsc.obj
 0001:00088684       WscScanTimeout             10089684 f   wsc.obj
 0001:000886e8       WscPINTimeout              100896e8 f   wsc.obj
 0001:000886ec       WscLEDTimer                100896ec f   wsc.obj
 0001:00088800       WscPushPBCAction           10089800 f   wsc.obj
 0001:00088910       WscPBCExec                 10089910 f   wsc.obj
 0001:00088ab0       WscSendMessageM8           10089ab0 f   wsc.obj
 0001:00089088       WscRecvMessageM4           1008a088 f   wsc.obj
 0001:00089414       WscRecvMessageM5           1008a414 f   wsc.obj
 0001:00089760       WscRecvMessageM6           1008a760 f   wsc.obj
 0001:00089aac       WscRecvMessageM7           1008aaac f   wsc.obj
 0001:00089e08       WscRecvMessageM8           1008ae08 f   wsc.obj
 0001:0008a080       WscEAPEnrolleeAction       1008b080 f   wsc.obj
 0001:0008a50c       WscEAPRegistrarAction      1008b50c f   wsc.obj
 0001:0008aa08       WscPBCTimeout              1008ba08 f   wsc.obj
 0001:0008aa48       WscEAPAction               1008ba48 f   wsc.obj
 0001:0008aad4       WscStateMachineInit        1008bad4 f   wsc.obj
 0001:0008ac8c       sha256_compile             1008bc8c f   wsc_crypto.obj
 0001:0008b87c       sha256_hash                1008c87c f   wsc_crypto.obj
 0001:0008ba74       sha256                     1008ca74 f   wsc_crypto.obj
 0001:0008bad8       hmac_sha_key               1008cad8 f   wsc_crypto.obj
 0001:0008bb7c       hmac_sha_data              1008cb7c f   wsc_crypto.obj
 0001:0008bc4c       hmac_sha_end               1008cc4c f   wsc_crypto.obj
 0001:0008bd4c       hmac_sha                   1008cd4c f   wsc_crypto.obj
 0001:0008bdc8       KD_hmac_sha256             1008cdc8 f   wsc_crypto.obj
 0001:0008be58       AES_encrypt                1008ce58 f   wsc_crypto.obj
 0001:0008c5bc       AES_decrypt                1008d5bc f   wsc_crypto.obj
 0001:0008cd1c       AES_set_encrypt_key        1008dd1c f   wsc_crypto.obj
 0001:0008d2b4       AES_cbc_encrypt            1008e2b4 f   wsc_crypto.obj
 0001:0008d59c       AES_set_decrypt_key        1008e59c f   wsc_crypto.obj
 0001:0008d7e8       EVP_EncryptInit            1008e7e8 f   wsc_crypto.obj
 0001:0008da04       EVP_EncryptUpdate          1008ea04 f   wsc_crypto.obj
 0001:0008db10       EVP_EncryptFinal           1008eb10 f   wsc_crypto.obj
 0001:0008db84       EVP_DecryptInit            1008eb84 f   wsc_crypto.obj
 0001:0008dbec       EVP_DecryptUpdate          1008ebec f   wsc_crypto.obj
 0001:0008dcc8       EVP_DecryptFinal           1008ecc8 f   wsc_crypto.obj
 0001:0008dd44       WscEncryptData             1008ed44 f   wsc_crypto.obj
 0001:0008de34       WscDecryptData             1008ee34 f   wsc_crypto.obj
 0001:0008df24       WscDeriveKey               1008ef24 f   wsc_crypto.obj
 0001:0008e090       NN_Decode                  1008f090 f   wsc_crypto.obj
 0001:0008e114       NN_Encode                  1008f114 f   wsc_crypto.obj
 0001:0008e184       NN_Sub                     1008f184 f   wsc_crypto.obj
 0001:0008e1f0       NN_LShift                  1008f1f0 f   wsc_crypto.obj
 0001:0008e24c       NN_RShift                  1008f24c f   wsc_crypto.obj
 0001:0008e2a8       NN_Cmp                     1008f2a8 f   wsc_crypto.obj
 0001:0008e300       NN_DigitMult               1008f300 f   wsc_crypto.obj
 0001:0008e370       NN_DigitDiv                1008f370 f   wsc_crypto.obj
 0001:0008e4c4       NN_Mult                    1008f4c4 f   wsc_crypto.obj
 0001:0008e678       NN_Div                     1008f678 f   wsc_crypto.obj
 0001:0008e944       NN_ModMult                 1008f944 f   wsc_crypto.obj
 0001:0008e98c       NN_ModExp                  1008f98c f   wsc_crypto.obj
 0001:0008eb48       GenerateDHPublicKey        1008fb48 f   wsc_crypto.obj
 0001:0008ec30       GenerateDHSecreteKey       1008fc30 f   wsc_crypto.obj
 0001:0008ed08       InitMDSMCtrl               1008fd08 f   tpc.obj
 0001:0008ed60       MDSMCalculateMaxTxPower    1008fd60 f   tpc.obj
 0001:0008ed7c       MDSMCreatePowerCapabilityIE 1008fd7c f   tpc.obj
 0001:0008edcc       MDSMCalaculateRealTxPower  1008fdcc f   tpc.obj
 0001:0008edec       RTMPCheckTDLSFrame         1008fdec f   tdls.obj
 0001:0008ee60       TDLSSendPacket             1008fe60 f   tdls.obj
 0001:0008f050       TdlsTimeout                10090050 f   tdls.obj
 0001:0008f0e0       TDLSSearchLinkId           100900e0 f   tdls.obj
 0001:0008f160       TPKMsg1Process             10090160 f   tdls.obj
 0001:0008f37c       TPKMsg3Process             1009037c f   tdls.obj
 0001:0008f71c       TDLSDeriveTPK              1009071c f   tdls.obj
 0001:0008f8c0       TDLSSearchTabInit          100908c0 f   tdls.obj
 0001:0008f9d4       TDLSSearchEntyAlloc        100909d4 f   tdls.obj
 0001:0008fa4c       TDLSSearchEntyFree         10090a4c f   tdls.obj
 0001:0008fabc       TLDSSearchEntryLookup      10090abc f   tdls.obj
 0001:0008fb54       TDLSSearchEntryUpdate      10090b54 f   tdls.obj
 0001:0008fc74       TDLSSearchEntryDelete      10090c74 f   tdls.obj
 0001:0008fd94       TDLSSearchTabMaintain      10090d94 f   tdls.obj
 0001:0008ff6c       TDLSLinkMaintenance        10090f6c f   tdls.obj
 0001:0009008c       TDLSDiscoveryPacketLearnAndCheck 1009108c f   tdls.obj
 0001:000901c4       MlmeTdlsSetupReqAction     100911c4 f   tdls.obj
 0001:0009099c       PeerTdlsSetupReqAction     1009199c f   tdls.obj
 0001:0009174c       PeerTdlsSetupConfAction    1009274c f   tdls.obj
 0001:000922bc       MlmeTdlsTearDownAction     100932bc f   tdls.obj
 0001:00092714       PeerTdlsTearDownAction     10093714 f   tdls.obj
 0001:00092aa4       RTMPSendTDLSTearDownFrame  10093aa4 f   tdls.obj
 0001:00092e74       TdlsTearDown               10093e74 f   tdls.obj
 0001:00093080       TPKMsg2Process             10094080 f   tdls.obj
 0001:00093434       TDLSTableInit              10094434 f   tdls.obj
 0001:0009348c       TDLSSearchTabDestory       1009448c f   tdls.obj
 0001:00093518       PeerTdlsSetupRspAction     10094518 f   tdls.obj
 0001:00094954       PeerTdlsMsgAction          10095954 f   tdls.obj
 0001:000949b8       TdlsStateMachineInit       100959b8 f   tdls.obj
 0001:00094aa0       EventModify                10095aa0 f   Coredll:COREDLL.dll
 0001:00094ab0       ExitThread                 10095ab0 f   Coredll:COREDLL.dll
 0001:00094ac0       WaitForSingleObject        10095ac0 f   Coredll:COREDLL.dll
 0001:00094ad0       CeSetThreadPriority        10095ad0 f   Coredll:COREDLL.dll
 0001:00094ae0       CreateThread               10095ae0 f   Coredll:COREDLL.dll
 0001:00094af0       CreateEventW               10095af0 f   Coredll:COREDLL.dll
 0001:00094b00       NKDbgPrintfW               10095b00 f   Coredll:COREDLL.dll
 0001:00094b10       InterlockedExchange        10095b10 f   Coredll:COREDLL.dll
 0001:00094b20       InterlockedDecrement       10095b20 f   Coredll:COREDLL.dll
 0001:00094b30       InterlockedIncrement       10095b30 f   Coredll:COREDLL.dll
 0001:00094b40       SetLastError               10095b40 f   Coredll:COREDLL.dll
 0001:00094b50       Sleep                      10095b50 f   Coredll:COREDLL.dll
 0001:00094b60       TerminateThread            10095b60 f   Coredll:COREDLL.dll
 0001:00094b70       GetExitCodeThread          10095b70 f   Coredll:COREDLL.dll
 0001:00094b80       RegCloseKey                10095b80 f   Coredll:COREDLL.dll
 0001:00094b90       RegQueryValueExW           10095b90 f   Coredll:COREDLL.dll
 0001:00094ba0       RegOpenKeyExW              10095ba0 f   Coredll:COREDLL.dll
 0001:00094bb0       GetSystemInfo              10095bb0 f   Coredll:COREDLL.dll
 0001:00094bc0       DisableThreadLibraryCalls  10095bc0 f   Coredll:COREDLL.dll
 0001:00094bd0       StringCbPrintfA            10095bd0 f   Coredll:COREDLL.dll
 0001:00094be0       NdisReleaseSpinLock        10095be0 f   ndis:NDIS.dll
 0001:00094bf0       NdisAcquireSpinLock        10095bf0 f   ndis:NDIS.dll
 0001:00094c00       NdisStallExecution         10095c00 f   ndis:NDIS.dll
 0001:00094c10       NdisGetSystemUpTime        10095c10 f   ndis:NDIS.dll
 0001:00094c20       NdisFreeMemory             10095c20 f   ndis:NDIS.dll
 0001:00094c30       NdisAllocateBuffer         10095c30 f   ndis:NDIS.dll
 0001:00094c40       NdisFreePacket             10095c40 f   ndis:NDIS.dll
 0001:00094c50       NdisAllocateMemoryWithTag  10095c50 f   ndis:NDIS.dll
 0001:00094c60       NdisAllocatePacket         10095c60 f   ndis:NDIS.dll
 0001:00094c70       NdisAllocateSpinLock       10095c70 f   ndis:NDIS.dll
 0001:00094c80       NdisFreeSpinLock           10095c80 f   ndis:NDIS.dll
 0001:00094c90       NdisMSleep                 10095c90 f   ndis:NDIS.dll
 0001:00094ca0       NdisInterlockedDecrement   10095ca0 f   ndis:NDIS.dll
 0001:00094cb0       NdisGetCurrentSystemTime   10095cb0 f   ndis:NDIS.dll
 0001:00094cc0       NdisQueryPacket            10095cc0 f   ndis:NDIS.dll
 0001:00094cd0       NdisAllocateBufferPool     10095cd0 f   ndis:NDIS.dll
 0001:00094ce0       NdisAllocatePacketPool     10095ce0 f   ndis:NDIS.dll
 0001:00094cf0       NdisInitializeNPagedLookasideList 10095cf0 f   ndis:NDIS.dll
 0001:00094d00       NdisDeleteNPagedLookasideList 10095d00 f   ndis:NDIS.dll
 0001:00094d10       NdisFreeBufferPool         10095d10 f   ndis:NDIS.dll
 0001:00094d20       NdisFreePacketPool         10095d20 f   ndis:NDIS.dll
 0001:00094d30       NdisMInitializeTimer       10095d30 f   ndis:NDIS.dll
 0001:00094d40       NdisSetTimer               10095d40 f   ndis:NDIS.dll
 0001:00094d50       NdisMSetPeriodicTimer      10095d50 f   ndis:NDIS.dll
 0001:00094d60       NdisMCancelTimer           10095d60 f   ndis:NDIS.dll
 0001:00094d70       NdisCloseConfiguration     10095d70 f   ndis:NDIS.dll
 0001:00094d80       NdisReadConfiguration      10095d80 f   ndis:NDIS.dll
 0001:00094d90       NdisOpenConfiguration      10095d90 f   ndis:NDIS.dll
 0001:00094da0       NdisUnicodeStringToAnsiString 10095da0 f   ndis:NDIS.dll
 0001:00094db0       NdisCloseFile              10095db0 f   ndis:NDIS.dll
 0001:00094dc0       NdisUnmapFile              10095dc0 f   ndis:NDIS.dll
 0001:00094dd0       NdisMapFile                10095dd0 f   ndis:NDIS.dll
 0001:00094de0       NdisOpenFile               10095de0 f   ndis:NDIS.dll
 0001:00094df0       NdisInitializeString       10095df0 f   ndis:NDIS.dll
 0001:00094e00       NdisMGetDeviceProperty     10095e00 f   ndis:NDIS.dll
 0001:00094e10       NdisMSetAttributesEx       10095e10 f   ndis:NDIS.dll
 0001:00094e20       NdisTerminateWrapper       10095e20 f   ndis:NDIS.dll
 0001:00094e30       NdisMRegisterMiniport      10095e30 f   ndis:NDIS.dll
 0001:00094e40       NdisInitializeWrapper      10095e40 f   ndis:NDIS.dll
 0001:00094e50       NdisInterlockedIncrement   10095e50 f   ndis:NDIS.dll
 0001:00094e60       NdisFreeBuffer             10095e60 f   ndis:NDIS.dll
 0001:00094e70       NdisUnchainBufferAtFront   10095e70 f   ndis:NDIS.dll
 0001:00094e80       NdisFreeToNPagedLookasideList 10095e80 f   ndis:NDIS.dll
 0001:00094e90       NdisAllocateFromNPagedLookasideList 10095e90 f   ndis:NDIS.dll
 0001:00094ea0       NdisDeregisterAdapter      10095ea0 f   ndis:NDIS.dll
 0001:00094eb0       NdisRegisterAdapter        10095eb0 f   ndis:NDIS.dll
 0001:00094ec0       RegisterClientSettings     10095ec0 f   usbd:USBD.dll
 0001:00094ed0       RegisterClientDriverID     10095ed0 f   usbd:USBD.dll
 0001:00094ee0       UnRegisterClientDriverID   10095ee0 f   usbd:USBD.dll
 0001:00094ef0       UnRegisterClientSettings   10095ef0 f   usbd:USBD.dll
 0001:00094f00       GetTransferStatus          10095f00 f   usbclient:usbclient.obj
 0001:00094f4c       IssueVendorTransfer        10095f4c f   usbclient:usbclient.obj
 0001:000950f4       ResetDefaultEndpoint       100960f4 f   usbclient:usbclient.obj
 0001:0009517c       ResetPipe                  1009617c f   usbclient:usbclient.obj
 0001:000951e0       __GSHandlerCheckCommon     100961e0 f   corelib0:gshandler.obj
 0001:0009521c       __GSHandlerCheck           1009621c f   corelib0:gshandler.obj
 0001:00095240       __security_check_cookie    10096240 f   corelib0:armsecgs.obj
 0001:00095254       __gsfailure                10096254 f   corelib0:armsecgs.obj
 0001:00095298       memcpy                     10096298 f   corelib1:COREDLL.dll
 0001:000952a8       memset                     100962a8 f   corelib1:COREDLL.dll
 0001:000952b8       strlen                     100962b8 f   corelib1:COREDLL.dll
 0001:000952c8       strcpy                     100962c8 f   corelib1:COREDLL.dll
 0001:000952d8       memmove                    100962d8 f   corelib1:COREDLL.dll
 0001:000952e8       __report_gsfailure         100962e8 f   corelib1:COREDLL.dll
 0001:000952f8       GetLastError               100962f8 f   Coredll:COREDLL.dll
 0001:000956a4       __IMPORT_DESCRIPTOR_COREDLL 100966a4     Coredll:COREDLL.dll
 0001:000956b8       __IMPORT_DESCRIPTOR_NDIS   100966b8     ndis:NDIS.dll
 0001:000956cc       __IMPORT_DESCRIPTOR_USBD   100966cc     usbd:USBD.dll
 0001:000956e0       __NULL_IMPORT_DESCRIPTOR   100966e0     Coredll:COREDLL.dll
 0002:00000000       __imp_EventModify          10097000     Coredll:COREDLL.dll
 0002:00000004       __imp_ExitThread           10097004     Coredll:COREDLL.dll
 0002:00000008       __imp_WaitForSingleObject  10097008     Coredll:COREDLL.dll
 0002:0000000c       __imp_CeSetThreadPriority  1009700c     Coredll:COREDLL.dll
 0002:00000010       __imp_CreateThread         10097010     Coredll:COREDLL.dll
 0002:00000014       __imp_CreateEventW         10097014     Coredll:COREDLL.dll
 0002:00000018       __imp_NKDbgPrintfW         10097018     Coredll:COREDLL.dll
 0002:0000001c       __imp_InterlockedExchange  1009701c     Coredll:COREDLL.dll
 0002:00000020       __imp_InterlockedDecrement 10097020     Coredll:COREDLL.dll
 0002:00000024       __imp_InterlockedIncrement 10097024     Coredll:COREDLL.dll
 0002:00000028       __imp_SetLastError         10097028     Coredll:COREDLL.dll
 0002:0000002c       __imp_Sleep                1009702c     Coredll:COREDLL.dll
 0002:00000030       __imp_TerminateThread      10097030     Coredll:COREDLL.dll
 0002:00000034       __imp_GetExitCodeThread    10097034     Coredll:COREDLL.dll
 0002:00000038       __imp_RegCloseKey          10097038     Coredll:COREDLL.dll
 0002:0000003c       __imp_RegQueryValueExW     1009703c     Coredll:COREDLL.dll
 0002:00000040       __imp_RegOpenKeyExW        10097040     Coredll:COREDLL.dll
 0002:00000044       __imp_GetSystemInfo        10097044     Coredll:COREDLL.dll
 0002:00000048       __imp_DisableThreadLibraryCalls 10097048     Coredll:COREDLL.dll
 0002:0000004c       __imp_StringCbPrintfA      1009704c     Coredll:COREDLL.dll
 0002:00000050       __imp___report_gsfailure   10097050     corelib1:COREDLL.dll
 0002:00000054       __imp_memmove              10097054     corelib1:COREDLL.dll
 0002:00000058       __imp_strcpy               10097058     corelib1:COREDLL.dll
 0002:0000005c       __imp_strlen               1009705c     corelib1:COREDLL.dll
 0002:00000060       __imp___rt_sdiv            10097060     corelib1:COREDLL.dll
 0002:00000064       __imp___rt_udiv            10097064     corelib1:COREDLL.dll
 0002:00000068       __imp_memset               10097068     corelib1:COREDLL.dll
 0002:0000006c       __imp_memcpy               1009706c     corelib1:COREDLL.dll
 0002:00000070       __imp_GetLastError         10097070     Coredll:COREDLL.dll
 0002:00000074       \177COREDLL_NULL_THUNK_DATA 10097074     Coredll:COREDLL.dll
 0002:00000078       __imp_NdisFreeSpinLock     10097078     ndis:NDIS.dll
 0002:0000007c       __imp_NdisMSleep           1009707c     ndis:NDIS.dll
 0002:00000080       __imp_NdisInterlockedDecrement 10097080     ndis:NDIS.dll
 0002:00000084       __imp_NdisGetCurrentSystemTime 10097084     ndis:NDIS.dll
 0002:00000088       __imp_NdisQueryPacket      10097088     ndis:NDIS.dll
 0002:0000008c       __imp_NdisAllocateBufferPool 1009708c     ndis:NDIS.dll
 0002:00000090       __imp_NdisAllocatePacketPool 10097090     ndis:NDIS.dll
 0002:00000094       __imp_NdisInitializeNPagedLookasideList 10097094     ndis:NDIS.dll
 0002:00000098       __imp_NdisDeleteNPagedLookasideList 10097098     ndis:NDIS.dll
 0002:0000009c       __imp_NdisFreeBufferPool   1009709c     ndis:NDIS.dll
 0002:000000a0       __imp_NdisAllocateSpinLock 100970a0     ndis:NDIS.dll
 0002:000000a4       __imp_NdisMInitializeTimer 100970a4     ndis:NDIS.dll
 0002:000000a8       __imp_NdisSetTimer         100970a8     ndis:NDIS.dll
 0002:000000ac       __imp_NdisMSetPeriodicTimer 100970ac     ndis:NDIS.dll
 0002:000000b0       __imp_NdisMCancelTimer     100970b0     ndis:NDIS.dll
 0002:000000b4       __imp_NdisCloseConfiguration 100970b4     ndis:NDIS.dll
 0002:000000b8       __imp_NdisReadConfiguration 100970b8     ndis:NDIS.dll
 0002:000000bc       __imp_NdisOpenConfiguration 100970bc     ndis:NDIS.dll
 0002:000000c0       __imp_NdisUnicodeStringToAnsiString 100970c0     ndis:NDIS.dll
 0002:000000c4       __imp_NdisCloseFile        100970c4     ndis:NDIS.dll
 0002:000000c8       __imp_NdisUnmapFile        100970c8     ndis:NDIS.dll
 0002:000000cc       __imp_NdisMapFile          100970cc     ndis:NDIS.dll
 0002:000000d0       __imp_NdisOpenFile         100970d0     ndis:NDIS.dll
 0002:000000d4       __imp_NdisInitializeString 100970d4     ndis:NDIS.dll
 0002:000000d8       __imp_NdisMGetDeviceProperty 100970d8     ndis:NDIS.dll
 0002:000000dc       __imp_NdisMSetAttributesEx 100970dc     ndis:NDIS.dll
 0002:000000e0       __imp_NdisTerminateWrapper 100970e0     ndis:NDIS.dll
 0002:000000e4       __imp_NdisMRegisterMiniport 100970e4     ndis:NDIS.dll
 0002:000000e8       __imp_NdisInitializeWrapper 100970e8     ndis:NDIS.dll
 0002:000000ec       __imp_NdisInterlockedIncrement 100970ec     ndis:NDIS.dll
 0002:000000f0       __imp_NdisFreeBuffer       100970f0     ndis:NDIS.dll
 0002:000000f4       __imp_NdisUnchainBufferAtFront 100970f4     ndis:NDIS.dll
 0002:000000f8       __imp_NdisFreeToNPagedLookasideList 100970f8     ndis:NDIS.dll
 0002:000000fc       __imp_NdisAllocateFromNPagedLookasideList 100970fc     ndis:NDIS.dll
 0002:00000100       __imp_NdisDeregisterAdapter 10097100     ndis:NDIS.dll
 0002:00000104       __imp_NdisRegisterAdapter  10097104     ndis:NDIS.dll
 0002:00000108       __imp_NdisReleaseSpinLock  10097108     ndis:NDIS.dll
 0002:0000010c       __imp_NdisAcquireSpinLock  1009710c     ndis:NDIS.dll
 0002:00000110       __imp_NdisStallExecution   10097110     ndis:NDIS.dll
 0002:00000114       __imp_NdisGetSystemUpTime  10097114     ndis:NDIS.dll
 0002:00000118       __imp_NdisFreeMemory       10097118     ndis:NDIS.dll
 0002:0000011c       __imp_NdisAllocatePacket   1009711c     ndis:NDIS.dll
 0002:00000120       __imp_NdisAllocateMemoryWithTag 10097120     ndis:NDIS.dll
 0002:00000124       __imp_NdisFreePacket       10097124     ndis:NDIS.dll
 0002:00000128       __imp_NdisAllocateBuffer   10097128     ndis:NDIS.dll
 0002:0000012c       __imp_NdisFreePacketPool   1009712c     ndis:NDIS.dll
 0002:00000130       \177NDIS_NULL_THUNK_DATA   10097130     ndis:NDIS.dll
 0002:00000134       __imp_UnRegisterClientDriverID 10097134     usbd:USBD.dll
 0002:00000138       __imp_RegisterClientDriverID 10097138     usbd:USBD.dll
 0002:0000013c       __imp_RegisterClientSettings 1009713c     usbd:USBD.dll
 0002:00000140       __imp_UnRegisterClientSettings 10097140     usbd:USBD.dll
 0002:00000144       \177USBD_NULL_THUNK_DATA   10097144     usbd:USBD.dll
 0002:00000474       CISCO_OUI                  10097474     aironet.obj
 0002:00000584       pEventText                 10097584     ap.obj
 0002:00000bfc       CipherSuiteWPAPSKTKIPLen   10097bfc     ap_info.obj
 0002:00000c00       APSupportedOids            10097c00     ap_info.obj
 0002:00000de8       CipherSuiteWPAPSKTKIP      10097de8     ap_info.obj
 0002:0000123c       CipherSuiteWAPIPsk         1009823c     Ap_wapi.obj
 0002:00001252       CipherSuiteWAPIPskLen      10098252     Ap_wapi.obj
 0002:00001253       CipherSuiteWAPICertLen     10098253     Ap_wapi.obj
 0002:00001254       CipherSuiteWAPICert        10098254     Ap_wapi.obj
 0002:0000126c       WAPI_PROTOTYPE             1009826c     Ap_wapi.obj
 0002:00001270       WAPI_INIT_PN               10098270     Ap_wapi.obj
 0002:00001404       OUI_WPA_WEP40              10098404     ap_wpa.obj
 0002:00001408       OUI_WPA_TKIP               10098408     ap_wpa.obj
 0002:0000140c       OUI_WPA_CCMP               1009840c     ap_wpa.obj
 0002:00001410       OUI_WPA2_WEP40             10098410     ap_wpa.obj
 0002:00001414       OUI_WPA2_TKIP              10098414     ap_wpa.obj
 0002:00001418       OUI_WPA2_CCMP              10098418     ap_wpa.obj
 0002:0000152c       CipherWpaTemplate          1009852c     assoc.obj
 0002:00001544       CipherWpaTemplateLen       10098544     assoc.obj
 0002:00001545       CipherWpa2TemplateLen      10098545     assoc.obj
 0002:00001548       CipherWpa2Template         10098548     assoc.obj
 0002:00001560       CcxVerIE                   10098560     assoc.obj
 0002:00001894       CipherSuiteWpaNoneTkip     10098894     connect.obj
 0002:000018aa       CipherSuiteWpaNoneTkipLen  100988aa     connect.obj
 0002:000018ab       CipherSuiteWpaNoneAesLen   100988ab     connect.obj
 0002:000018ac       CipherSuiteWpaNoneAes      100988ac     connect.obj
 0002:00001ae4       SNAP_LEAP_ROGUEAP_HDR      10098ae4     leap.obj
 0002:00001c00       PADDING                    10098c00     md4.obj
 0002:00004684       RateSwitchTable11B         1009b684     mlme.obj
 0002:0000469d       SupRateIe                  1009b69d     mlme.obj
 0002:0000469e       ExtRateIe                  1009b69e     mlme.obj
 0002:0000469f       HtCapIe                    1009b69f     mlme.obj
 0002:000046a0       RateSwitchTable            1009b6a0     mlme.obj
 0002:00004745       AddHtInfoIe                1009b745     mlme.obj
 0002:00004746       NewExtChanIe               1009b746     mlme.obj
 0002:00004747       ExtHtCapIe                 1009b747     mlme.obj
 0002:00004748       RateSwitchTable11BG        1009b748     mlme.obj
 0002:0000477f       ErpIe                      1009b77f     mlme.obj
 0002:00004780       RateSwitchTable11G         1009b780     mlme.obj
 0002:000047ad       DsIe                       1009b7ad     mlme.obj
 0002:000047ae       TimIe                      1009b7ae     mlme.obj
 0002:000047af       WpaIe                      1009b7af     mlme.obj
 0002:000047b0       RateSwitchTable11N1S       1009b7b0     mlme.obj
 0002:000047f1       Wpa2Ie                     1009b7f1     mlme.obj
 0002:000047f2       IbssIe                     1009b7f2     mlme.obj
 0002:000047f3       CcxIe                      1009b7f3     mlme.obj
 0002:000047f4       RateSwitchTable11N2SForABand 1009b7f4     mlme.obj
 0002:00004830       RateSwitchTable11N2S       1009b830     mlme.obj
 0002:0000487b       BssIntRepIe                1009b87b     mlme.obj
 0002:0000487c       RateSwitchTable11BGN2SForABand 1009b87c     mlme.obj
 0002:000048b8       RateSwitchTable11BGN1S     1009b8b8     mlme.obj
 0002:000048f9       BssCoexistIe               1009b8f9     mlme.obj
 0002:00004900       RateSwitchTable11BGN2S     1009b900     mlme.obj
 0002:00004950       ReasonString               1009b950     mlme.obj
 0002:00004998       BasicRateMask              1009b998     mlme.obj
 0002:000049c8       MULTICAST_ADDR             1009b9c8     mlme.obj
 0002:000049d0       BROADCAST_ADDR             1009b9d0     mlme.obj
 0002:000049d8       RssiSafeLevelForTxRate     1009b9d8     mlme.obj
 0002:000049e8       Phy11BNextRateDownward     1009b9e8     mlme.obj
 0002:000049ec       Phy11BNextRateUpward       1009b9ec     mlme.obj
 0002:000049f0       Phy11BGNextRateDownward    1009b9f0     mlme.obj
 0002:000049fc       Phy11BGNextRateUpward      1009b9fc     mlme.obj
 0002:00004a08       Phy11ANextRateDownward     1009ba08     mlme.obj
 0002:00004a14       Phy11ANextRateUpward       1009ba14     mlme.obj
 0002:00004a20       RateUpPER                  1009ba20     mlme.obj
 0002:00004a38       RateDownPER                1009ba38     mlme.obj
 0002:00004a50       RateIdToMbps               1009ba50     mlme.obj
 0002:00004a60       RateIdTo500Kbps            1009ba60     mlme.obj
 0002:00004a7c       SES_OUI                    1009ba7c     mlme.obj
 0002:00004a80       RateOFDMToCCK              1009ba80     mlme.obj
 0002:00004a88       RF2850RegTable             1009ba88     mlme.obj
 0002:00004f38       FreqItems3020              1009bf38     mlme.obj
 0002:00004f70       FreqItems3572              1009bf70     mlme.obj
 0002:00005044       AntStr                     1009c044     mlme.obj
 0002:00005054       NIC_VENDOR_DESC            1009c054     oem.obj
 0002:00005070       NIC_VENDOR_DESC_LEN        1009c070     oem.obj
 0002:00005074       NIC_WPS_DESC               1009c074     oem.obj
 0002:00005084       NIC_WPS_DESC_LEN           1009c084     oem.obj
 0002:00005088       NIC_VENDOR_DRIVER_VERSION  1009c088     oem.obj
 0002:0000508c       LINKNAME_STRING            1009c08c     oem.obj
 0002:000050b4       NTDEVICE_STRING            1009c0b4     oem.obj
 0002:00005408       Wpa2AuthEncryptPairs       1009c408     rtmp_info.obj
 0002:00005478       ralinkrate                 1009c478     rtmp_info.obj
 0002:00005678       STASupportedOids           1009c678     rtmp_info.obj
 0002:00005ad4       BIT8                       1009cad4     rtmp_init.obj
 0002:00005ae0       BIT32                      1009cae0     rtmp_init.obj
 0002:00005b60       CipherName                 1009cb60     rtmp_init.obj
 0002:00005b80       NICRegTable                1009cb80     rtmp_init.obj
 0002:00006750       BBPRegTable                1009d750     rtmp_init.obj
 0002:00006770       RFRegTable                 1009d770     rtmp_init.obj
 0002:00006798       RF3572RegTable             1009d798     rtmp_init.obj
 0002:000067d8       RF3320RegTable             1009d7d8     rtmp_init.obj
 0002:00006818       TxPowerTuningTable         1009d818     rtmp_init.obj
 0002:000068b0       MACRegTable                1009d8b0     rtmp_init.obj
 0002:000069a0       FirmwareImage              1009d9a0     rtmp_init.obj
 0002:000074d0       FirmwareV2Image            1009e4d0     rtmp_init.obj
 0002:0000810c       RTDebugLevel               1009f10c     rtmp_main.obj
 0002:00008220       Tkip_Sbox_Lower            1009f220     rtmp_tkip.obj
 0002:00008620       Tkip_Sbox_Upper            1009f620     rtmp_tkip.obj
 0002:0000914c       EpToQueue                  100a014c     rtusb_bulk.obj
 0002:00009154       AMSDUPadShift              100a0154     rtusb_bulk.obj
 0002:00009274       SNAP_802_1H                100a0274     rtusb_data.obj
 0002:0000927c       SNAP_BRIDGE_TUNNEL         100a027c     rtusb_data.obj
 0002:00009284       SNAP_AIRONET               100a0284     rtusb_data.obj
 0002:0000928c       CKIP_LLC_SNAP              100a028c     rtusb_data.obj
 0002:00009294       AIRONET_PROTOCOL           100a0294     rtusb_data.obj
 0002:00009298       EAPOL_LLC_SNAP             100a0298     rtusb_data.obj
 0002:000092a0       WAI_LLC_SNAP               100a02a0     rtusb_data.obj
 0002:000092a8       EAPOL                      100a02a8     rtusb_data.obj
 0002:000092ac       IPX                        100a02ac     rtusb_data.obj
 0002:000092b0       APPLE_TALK                 100a02b0     rtusb_data.obj
 0002:000092b4       RateIdToPlcpSignal         100a02b4     rtusb_data.obj
 0002:000092c0       OfdmSignalToRateId         100a02c0     rtusb_data.obj
 0002:000092d0       OfdmRateToRxwiMCS          100a02d0     rtusb_data.obj
 0002:000092dc       RxwiMCSToOfdmRate          100a02dc     rtusb_data.obj
 0002:000092e8       MCSToMbps                  100a02e8     rtusb_data.obj
 0002:00009308       default_cwmin              100a0308     rtusb_data.obj
 0002:0000930c       default_cwmax              100a030c     rtusb_data.obj
 0002:00009310       default_sta_aifsn          100a0310     rtusb_data.obj
 0002:00009314       MapUserPriorityToAccessCategory 100a0314     rtusb_data.obj
 0002:0000953c       WPA_OUI                    100a053c     sanity.obj
 0002:00009540       RSN_OUI                    100a0540     sanity.obj
 0002:00009544       WPS_OUI                    100a0544     sanity.obj
 0002:00009548       WME_INFO_ELEM              100a0548     sanity.obj
 0002:00009550       WME_PARM_ELEM              100a0550     sanity.obj
 0002:00009558       RALINK_OUI                 100a0558     sanity.obj
 0002:0000955c       PRE_N_HT_OUI               100a055c     sanity.obj
 0002:00009560       SSIDL_OUI                  100a0560     sanity.obj
 0002:00009674       WAIHEAD                    100a0674     Sta_wapi.obj
 0002:0000967c       WAPI_INIT_SEQ              100a067c     Sta_wapi.obj
 0002:0000978c       A_BAND_REGION_0_CHANNEL_LIST 100a078c     sync.obj
 0002:0000979c       A_BAND_REGION_1_CHANNEL_LIST 100a079c     sync.obj
 0002:000097b0       A_BAND_REGION_2_CHANNEL_LIST 100a07b0     sync.obj
 0002:000097b8       A_BAND_REGION_3_CHANNEL_LIST 100a07b8     sync.obj
 0002:000097c0       A_BAND_REGION_4_CHANNEL_LIST 100a07c0     sync.obj
 0002:000097c8       A_BAND_REGION_5_CHANNEL_LIST 100a07c8     sync.obj
 0002:000097cc       A_BAND_REGION_6_CHANNEL_LIST 100a07cc     sync.obj
 0002:000097d0       A_BAND_REGION_7_CHANNEL_LIST 100a07d0     sync.obj
 0002:000097e8       A_BAND_REGION_8_CHANNEL_LIST 100a07e8     sync.obj
 0002:000097ec       A_BAND_REGION_9_CHANNEL_LIST 100a07ec     sync.obj
 0002:00009804       A_BAND_REGION_10_CHANNEL_LIST 100a0804     sync.obj
 0002:00009810       A_BAND_REGION_11_CHANNEL_LIST 100a0810     sync.obj
 0002:00009824       A_BAND_REGION_12_CHANNEL_LIST 100a0824     sync.obj
 0002:00009838       A_BAND_REGION_13_CHANNEL_LIST 100a0838     sync.obj
 0002:0000984c       A_BAND_REGION_14_CHANNEL_LIST 100a084c     sync.obj
 0002:00009860       A_BAND_REGION_15_CHANNEL_LIST 100a0860     sync.obj
 0002:00009868       A_BAND_REGION_16_CHANNEL_LIST 100a0868     sync.obj
 0002:00009884       BaSizeArray                100a0884     sync.obj
 0002:00009998       SupportedDev               100a0998     wince.obj
 0002:00009d44       CipherWpaPskTkip           100a0d44     wpa.obj
 0002:00009d5c       CipherWpaPskTkipLen        100a0d5c     wpa.obj
 0002:00009d5d       CipherWpaPskAesLen         100a0d5d     wpa.obj
 0002:00009d5e       CipherSuiteCiscoCCKMLen    100a0d5e     wpa.obj
 0002:00009d5f       CipherSuiteCiscoCCKMWPALen 100a0d5f     wpa.obj
 0002:00009d60       CipherWpaPskAes            100a0d60     wpa.obj
 0002:00009d78       CipherSuiteCiscoCCKMCKIP   100a0d78     wpa.obj
 0002:00009d90       CipherSuiteCiscoCCKMCkipCmic 100a0d90     wpa.obj
 0002:00009da8       CipherSuiteCiscoCCKMCmic   100a0da8     wpa.obj
 0002:00009dc0       CipherSuiteCiscoCCKMWep40  100a0dc0     wpa.obj
 0002:00009dd8       CipherSuiteCiscoCCKMWep104 100a0dd8     wpa.obj
 0002:00009df0       CipherSuiteCiscoCCKMTkip   100a0df0     wpa.obj
 0002:00009e08       CipherSuiteCiscoCCKMAES    100a0e08     wpa.obj
 0002:00009e20       CipherSuiteCiscoCCKMTkip24 100a0e20     wpa.obj
 0002:00009e3a       CipherSuiteCiscoCCKMTkip24Len 100a0e3a     wpa.obj
 0002:00009e3b       CipherSuiteCCXTkipLen      100a0e3b     wpa.obj
 0002:00009e3c       CipherSuiteCCXTkip         100a0e3c     wpa.obj
 0002:00009e54       CipherSuiteCiscoCCKMWPA2Tkip 100a0e54     wpa.obj
 0002:00009e6a       CipherSuiteCiscoCCKMWPA2Len 100a0e6a     wpa.obj
 0002:00009e6c       CipherSuiteCiscoCCKMWPA2AES 100a0e6c     wpa.obj
 0002:00009f94       Wsc_Uuid                   100a0f94     wsc.obj
 0002:00009fa4       Wsc_Manufacture            100a0fa4     wsc.obj
 0002:00009fc0       Wsc_Model_Name             100a0fc0     wsc.obj
 0002:00009fd8       Wsc_Model_Number           100a0fd8     wsc.obj
 0002:00009fe0       Wsc_Model_Serial           100a0fe0     wsc.obj
 0002:00009fec       Wsc_Pri_Dev_Type           100a0fec     wsc.obj
 0002:00009ff4       Wsc_Dev_Name_R             100a0ff4     wsc.obj
 0002:0000a008       Wsc_Personal_String        100a1008     wsc.obj
 0002:0000a030       EnrolleeMsg                100a1030     wsc.obj
 0002:0000a050       RegistrarMsg               100a1050     wsc.obj
 0002:0000a070       THOME_303V_MODEL_NAME      100a1070     wsc.obj
 0002:0000a07c       THOME_303V_MODEL_NUMBER_000 100a107c     wsc.obj
 0002:0000a088       THOME_303V_MODEL_NUMBER_001 100a1088     wsc.obj
 0002:0000a374       dot11dhCountry             100a1374     tpc.obj
 0002:0000a375       dot11dhHoppingPatternParameters 100a1375     tpc.obj
 0002:0000a376       dot11dhHoppingPatternTable 100a1376     tpc.obj
 0002:0000a377       dot11dhRequest             100a1377     tpc.obj
 0002:0000a378       dot11dhPowerConstraint     100a1378     tpc.obj
 0002:0000a379       dot11dhPowerCapability     100a1379     tpc.obj
 0002:0000a37a       dot11dhTPCRequest          100a137a     tpc.obj
 0002:0000a37b       dot11dhTPCReport           100a137b     tpc.obj
 0002:0000a37c       dot11dhSupportedChannel    100a137c     tpc.obj
 0002:0000a37d       dot11dhChannelSwitchAnnouncement 100a137d     tpc.obj
 0002:0000a37e       dot11dhMeasurementRequest  100a137e     tpc.obj
 0002:0000a37f       dot11dhMeasurementReport   100a137f     tpc.obj
 0002:0000a380       dot11dhQuiet               100a1380     tpc.obj
 0002:0000a381       dot11dhIbssDFS             100a1381     tpc.obj
 0002:0000a494       TDLS_LLC_SNAP              100a1494     tdls.obj
 0002:0000a49c       TDLS_LLC_SNAP_WITH_CATEGORY 100a149c     tdls.obj
 0002:0000a4a6       LinkIdIe                   100a14a6     tdls.obj
 0002:0000a4a7       QosCapIe                   100a14a7     tdls.obj
 0002:0000a4a8       TDLS_ETHERTYPE             100a14a8     tdls.obj
 0002:0000a4aa       FastTransIe                100a14aa     tdls.obj
 0002:0000a4ab       TimeoutIntIe               100a14ab     tdls.obj
 0002:0000a4ac       CipherSuiteTDLSWpa2PskTkip 100a14ac     tdls.obj
 0002:0000a4c2       CipherSuiteTDLSLen         100a14c2     tdls.obj
 0002:0000a4c4       CipherSuiteTDLSWpa2PskAes  100a14c4     tdls.obj
 0002:0000a4dc       __security_cookie          100a14dc     corelib0:seccinit.obj
 0002:0000a4e0       __security_cookie_complement 100a14e0     corelib0:seccinit.obj
 0002:0000b508       desiredTSSIOverCCK         100a2508     mlme.obj
 0002:0000b50c       desiredTSSIOverOFDM        100a250c     mlme.obj
 0002:0000b514       desiredTSSIOverHT          100a2514     mlme.obj
 0002:0000b51c       desiredTSSIOverHTUsingSTBC 100a251c     mlme.obj
 0002:0000b524       ZERO_MAC_ADDR              100a2524     mlme.obj
 0002:0000b52a       SsidIe                     100a252a     mlme.obj
 0002:0000b52c       ZeroSsid                   100a252c     mlme.obj
 0002:0000b580       PlainText                  100a2580     <common>
 0002:0000bb60       CipherText                 100a2b60     <common>
 0002:0000c140       HmacData                   100a3140     <common>
 0002:0000d140       OutMsgBuf                  100a4140     <common>
 0002:0000dcf8       GUsbFuncs                  100a4cf8     <common>
 0002:0000dcfc       GhDevice                   100a4cfc     <common>
 0002:0000dd00       GUsbInterface              100a4d00     <common>
 0002:0000dd20       LocalStrings               100a4d20     <common>

 entry point at        0001:00080404

 Static symbols

 0001:00035580       SHAHashBlock               10036580 f   md5.obj
 0001:0008b93c       sha_end1                   1008c93c f   wsc_crypto.obj
